:100000000C94970B0C9464410C94C4410C94B40B65
:100010000C94B40B0C94B40B0C94CE410C94B40B14
:100020000C94B40B0C94D8410C94B40B0C94B40BFA
:100030000C94B40B0C94B40B0C94B40B0C94B40B44
:100040000C943E420C94B40B0C94B40B0C94B40B73
:100050000C9464420C948B420C94BA420C94B40BF2
:100060000C94B40B0C94B40B0C94B40B0C94B40B14
:100070000C94B40B0C94B40B0C94B40B312E32369C
:100080002E30300017151515151517001212121203
:10009000121212001711111714141700171111174B
:1000A0001111170015151517111111001714141738
:1000B0001111170017141417151517000000000070
:1000C0000000000084008C0094009C00A400AC00A0
:1000D000B400BC004845414400474554202F00521D
:1000E00045424F4F540D0A0052455345540D0A00E6
:1000F0004A4A59004750530054532D4E5450303102
:100100005F585858585858006E74702E6A73742E81
:100110006D666565642E61642E6A70003030302E25
:100120003030302E3030302E303030003030302E05
:100130003030302E3030302E303030003030302EF5
:100140003030302E3030302E3030300008011C017D
:100150002C013C018C07AC07CC07EC073031323363
:1001600034353637383941424344454600485454C3
:10017000502F312E312032303020485454500D0A47
:10018000436F6E6E656374696F6E3A20636C6F7354
:10019000650D0A436F6E74656E742D547970653AFF
:1001A00020746578742F68746D6C0D0A4361636800
:1001B000652D436F6E74726F6C3A206E6F2D6361A4
:1001C0006368650D0A436F6E74656E742D4C616EC5
:1001D00067756167653A20656E0D0A0D0A0048541F
:1001E00054502F312E3120323030204F4B0D0A43E6
:1001F0006F6E6E656374696F6E3A20636C6F7365C2
:100200000D0A436F6E74656E742D547970653A20D3
:10021000746578742F68746D6C0D0A43616368654A
:100220002D436F6E74726F6C3A206E6F2D63616335
:1002300068650D0A436F6E74656E742D4C616E6750
:10024000756167653A20656E0D0A0D0A3C21444FC1
:1002500043545950452048544D4C205055424C4928
:100260004320222D2F2F5733432F2F44544420480F
:10027000544D4C20342E3031205472616E736974A9
:10028000696F6E616C2F2F454E2220226874747046
:100290003A2F2F7777772E77332E6F72672F54523E
:1002A0002F68746D6C342F6C6F6F73652E6474647B
:1002B000223E3C48544D4C3E3C484541443E3C5413
:1002C00049544C453E54532D4E54502D534552568F
:1002D00045522053455455503C2F5449544C453EAB
:1002E0003C2F484541443E3C424F445920424743FD
:1002F0004F4C4F523D2223464646464646464622EE
:100300003E3C43454E5445523E3C423E00223E3C1C
:100310002F464F524D3E3C42523E3C464F4E54209B
:10032000434F4C4F523D22475245454E223E564187
:100330004C55452053415645443C2F464F4E543E64
:100340003C42523E00223E3C42523E3C42523E3CE7
:10035000494E50555420545950453D225355424D15
:100360004954222056414C55453D224150504C594C
:10037000223E3C2F464F524D3E004950004E4D000C
:10038000475700444E004243007A037D03800383B5
:100390000386032000240028002C00C0006401A86C
:1003A000C000FFFFFF0101A8C00101A8C0FF01A814
:1003B000C049502041444452455353005355424E86
:1003C0004554204D41534B00474154455741590036
:1003D000444E5320534552564552004144445245E1
:1003E000535300B103BC03C803D003DB034E3100F9
:1003F0004E32004E33004E3400ED03F003F303F6AB
:1004000003534552564552310053455256455232D8
:1004100000534552564552330053455256455234C7
:10042000000104090411041904400060008000A0C8
:100430000000504F574552204F4E004558544552EA
:100440004E414C2052455345540042524F574E2086
:100450004F55542052455345540057415443484446
:100460004F472054494D455220524553455400456D
:100470004E4332384A36302052454345495645208E
:100480004552524F5200415250205245515545530A
:10049000542054494D454F5554204552524F520017
:1004A00049434D50205041434B4554204348454318
:1004B0004B2053554D204552524F5200544350202B
:1004C0005041434B455420434845434B2053554DE1
:1004D000204552524F5200554450205041434B4505
:1004E0005420434845434B2053554D204552524FCD
:1004F000520049434D50204D455353414745004418
:100500004843502052454345495645204E414B28CB
:1005100052455452592900444843502052454E45B3
:1005200057414C20535441544500444843502052B5
:100530004542494E44205354415445004448435099
:100540002045585049524544205354415445004495
:100550004843502052454345495645205041434B5E
:100560004554204552524F52004E4254205245436A
:1005700045495645204552524F52004E425420465E
:100580004F524D4154204552524F52004E4254203A
:100590005041434B4554204552524F52004E425415
:1005A0002054494D45204F555428534552564552E5
:1005B0003129004E42542054494D45204F5554286E
:1005C0005345525645523229004E42542054494D0B
:1005D00045204F5554285345525645523329004E15
:1005E00042542054494D45204F55542853455256A6
:1005F0004552342900444E532054494D45204F550F
:100600005428534552564552312900444E532054E4
:10061000494D45204F55542853455256455232298D
:1006200000444E532054494D45204F5554285345BE
:1006300052564552332900444E532054494D4520CB
:100640004F5554285345525645523429004E545064
:1006500020554E53594E43524F4E495A4544004E31
:1006600054502054494D45204F5554285345525617
:1006700045523129004E54502054494D45204F5584
:1006800054285345525645523229004E5450205456
:10069000494D45204F55542853455256455233290C
:1006A000004E54502054494D45204F555428534531
:1006B000525645523429004E545020494C4C45471F
:1006C000414C20534552564552205245504C5900FA
:1006D0004E5450204C454150205345434F4E4420EA
:1006E00041444A5553540054494D4520494C4C45CA
:1006F00047414C00475053204E4D454120464F52F4
:100700004D4154204552524F52004E4D45412043D9
:100710004845434B53554D204552524F5200544982
:100720004D452044415441205245434549564520BA
:100730004552524F5200554E53594E432054494D45
:1007400045555000310432043B044A045A046F04F6
:100750008604A004BC04D704F204FF0417052A058C
:100760003C054F0569057B058C059D05B305C9054D
:10077000DF05F5050B06210637064D065F067506F3
:100780008B06A106B706D006E706F4060A071E0781
:1007900036076E772E636769006E732E6367690094
:1007A0006E622E63676900636C2E63676900656C17
:1007B0002E6367690073642E6367690066617669FA
:1007C000636F0092079907A007A707AE07B507BC9C
:1007D00007464958204E4554574F524B20534554D5
:1007E00054494E470054494D4520534552564552B1
:1007F0002053455454494E470054494D45205052CA
:100800004F564944452053455454494E4700544996
:100810004D452042524F414443415354204C4F4791
:10082000004556454E54204C4F47005359535445AC
:100830004D20494E464F4D4154494F4E00D107E59A
:1008400007F9070E0821082B084E54502041444A4E
:100850005553544D454E54204D4F44450042524F40
:100860004144434153542041444A5553544D454E0D
:1008700054204D4F4445004750532041444A55535E
:10088000544D454E54204D4F4445004A4A5920434B
:100890004C4F434B2041444A5553544D454E5420F0
:1008A0004D4F44450049085D0877088B084E4F209E
:1008B000414C41524D2854494D452053594E4352C5
:1008C0004F4E495A4544290054494D4520414C4119
:1008D000524D284E4F542053594E43524F4E495A71
:1008E0004544290054494D4520554E41444A5553ED
:1008F0005445440054494D45204F504552415449B8
:100900004F4E2054494D454F555400465552554E73
:100910004F20525443204D4F444500465552554EAA
:100920004F20475053204D4F444500555443204DD0
:100930004F44452856414C494429005554432050C2
:1009400050534F5554204D4F44452856414C49442F
:100950002900554E49564750532054494D45204E85
:100960004F2056414C4944004E4F2054494D45209C
:10097000494E50555400AD08C808E408F4080B0966
:100980001B092B093B095209680920485454502F70
:10099000003C2F413E3C42523E003F223E003C4242
:1009A000523E3C4120485245463D222E2F00545392
:1009B0002D4E54502D5345525645523C2F423E3CED
:1009C00042523E004243004954424C00223E3C42C7
:1009D000523E3C42523E494E54455256414C285399
:1009E00065632E2030206F72203E3635353334203B
:1009F00049676E6F7265293C42523E3C494E5055E4
:100A00005420545950453D225445585422204E41BB
:100A10004D453D224954424C222053495A453D22DE
:100A20003822204D41584C454E4754483D223522EE
:100A30002056414C55453D22003530223E3C2F5436
:100A4000483E3C54482057494454483D22313530B3
:100A5000223E54494D453C2F54483E3C5448205773
:100A6000494454483D22313530223E414D4F554E88
:100A7000543C2F54483E3C54482057494454483D28
:100A800022313530223E4E4F54453C2F54483E3C97
:100A90002F54523E003C2F54443E3C2F54523E00B3
:100AA0003C2F54443E3C54443E26656D73703B00DD
:100AB0003C2F54443E3C54443E42432041444A551A
:100AC0005354006D732E007365632C006F7665724E
:100AD0002039686F7572732E00444953545249424D
:100AE0005554494F4E002D2D2D2D2D3C2F54443E55
:100AF0003C54443E003C2F54443E3C54443E00266B
:100B0000656D73703B003C2F54443E3C54443E00A2
:100B10003C545220414C49474E3D2243454E54459A
:100B200052223E3C54443E004552525253540043DC
:100B30004C520050473D3100313530223E54494D32
:100B4000453C2F54483E3C54482057494454483D66
:100B500022353030223E4556454E543C2F54483EB7
:100B60003C2F54523E003C2F54443E3C2F54523EA6
:100B70000026656D73703B3C2F54443E3C54443E0C
:100B800026656D73703B002C44415441313A002C72
:100B9000434F44453A0028545950453A002C4E459D
:100BA00058543A002C434E543A00285354533A00B8
:100BB0003C2F54443E3C54443E002D2D2D2D2F2DD2
:100BC0002D2F2D2D202D2D3A2D2D3A2D2D003C543D
:100BD0005220414C49474E3D2243454E54455222F6
:100BE0003E3C54443E003C2F5441424C453E3C4226
:100BF000523E004F5045524154494E472054494DB2
:100C000045004D494E2E00484F555220004649524E
:100C10004D574152452056455253494F4E00454E7F
:100C20004332384A3630205245564953494F4E00D8
:100C30004D414320414444524553530054494D458E
:100C400020535441545553004F5045524154494F3D
:100C50004E204D4F4445004E455442494F53204E7F
:100C6000414D4500444E532053455256455200478E
:100C70004154455741592041444452455353005330
:100C800055424E4554204D41534B0049502041445C
:100C9000445245535300323030223E4954454D3C76
:100CA0002F54483E3C54482057494454483D223331
:100CB0003030223E56414C55453C2F54483E3C2F47
:100CC00054523E003C2F54443E3C2F54523E003C74
:100CD0002F54443E3C54443E003C545220414C4925
:100CE000474E3D2243454E544552223E3C54443EDD
:100CF00000222056414C55453D220022204D4158AE
:100D00004C454E4754483D2200222053495A453D08
:100D100022003C42523E3C494E50555420545950BA
:100D2000453D225445585422204E414D453D220018
:100D3000223E3C42523E003C42523E3C2F43454EF6
:100D40005445523E3C2F424F44593E3C2F48544D4F
:100D50004C3E003C42523E3C4120485245463D22DA
:100D60002E2F223E4D41494E204D454E553C2F41A0
:100D70003E3C42523E003C42523E003F455252529F
:100D80005354223E4552524F52204F46463C2F412B
:100D90003E3C42523E0026656D73703B3C4120480C
:100DA0005245463D22003F434C52223E4C4F472085
:100DB000434C4541523C2F413E003F50473D31227C
:100DC0003E5B325D3C2F413E26656D73703B3C417E
:100DD00020485245463D22003F50473D30223E5B71
:100DE000315D3C2F413E26656D73703B3C41204890
:100DF0005245463D22003C2F5441424C453E3C4228
:100E0000523E3C4120485245463D22003C2F423E46
:100E10003C42523E3C42523E3C5441424C452042B0
:100E20004F524445523D2231223E3C54523E3C54A6
:100E3000482057494454483D220022204D455448FB
:100E40004F443D22474554003C2F423E3C42523ED7
:100E50003C464F524D20414354494F4E3D22005392
:100E6000554E004D4F4E00545545005745440054D3
:100E70004855004652490053415400414955545287
:100E8000475550564E54532D4E54502D534552569F
:100E90004552303100454E4332384A3630205245B3
:100EA000563A00494E495449414C495A494E472EF9
:100EB0002E2E00494E495449414C495A4544004B55
:100EC0004559494E50555420494C4C4547414C00DA
:100ED0004D544B3333333920494E49542E2E2E0076
:100EE00043414C2052454D3A004448435020444928
:100EF0005341424C4544004448435020454E4142F2
:100F00004C4544004E545020525820454E41424CCE
:100F10004544004E54502052582044495341424CBD
:100F200045440042524F414443415354204C4F47A3
:100F3000004F5045524154494E472054494D4500B9
:100F4000475053204D4F4445205245414459004A93
:100F50004A59204D4F444520524541445900465579
:100F600052554E4F20475053204D4F444500554E4B
:100F7000495620475053204D4F444500454E43327B
:100F8000384A363020494E495445525200850E9514
:100F90000EA30EB30EBF0ED00EE00EE90EF70E0438
:100FA0000F130F230F310F400F4F0F5E0F6E0F7C8B
:100FB0000F56657273696F6E00504C454153452062
:100FC000434845434B204B455900504C4541534500
:100FD000205245534554004D41433A004448435044
:100FE000434E543A004E42432052454D3A00574139
:100FF000495420666F722054494D45205258004391
:101000004F4E4E4543542054532D4A4A59303200D6
:10101000434845434B204349524355495400504CA3
:1010200045415345205741495400434845434B20CF
:10103000434F4E4E4543544F5200B10FB90FCA0FA4
:10104000D70FDC0FE50FEE0FFF0F10101E102A1048
:1010500045585049524544200020524542494E448B
:10106000200052454E4557414C2000494E46494EBE
:10107000495459005010591062106B104A535400D3
:101080004B535400434354005554430050535400B1
:10109000484454007C108010841088108C109010EC
:1010A0002020202020202020202020202020202040
:1010B00000504F574552204F4E0045585445524E10
:1010C000414C2052455345540042524F574E204FF9
:1010D0005554205245534554005741544348444FBA
:1010E0004720524553455400454E43205243562015
:1010F0004552524F520041525020524551205449BE
:101100004D454F55540049434D502053554D2045B2
:1011100052524F52005443502053554D2045525285
:101120004F52005544502053554D204552524F5276
:101130000049434D50204D455353414745205243AC
:101140005600444843502052454345495645204E99
:10115000414B00444843502052454E4557414C00B6
:101160004448435020524542494E4400444843506D
:10117000204558504952454400444843502050436C
:1011800054204552524F52004E4254205243562052
:101190004552524F52004E425420464F524D4154F8
:1011A000204552524F52004E4254205041434B452D
:1011B00054204552524F52004E42542054494D45FE
:1011C0004F5554284E6F3129004E42542054494DFA
:1011D000454F5554284E6F3229004E4254205449F1
:1011E0004D454F5554284E6F3329004E42542054DC
:1011F000494D454F5554284E6F342900444E5320D5
:1012000054494D454F5554284E6F312900444E5393
:101210002054494D454F5554284E6F322900444EB5
:10122000532054494D454F5554284E6F332900449F
:101230004E532054494D454F5554284E6F34290084
:101240004E545020554E53594E43524F4E495A45D5
:10125000004E54502054494D454F5554284E6F313F
:1012600029004E54502054494D454F5554284E6F37
:101270003229004E54502054494D454F5554284E64
:101280006F3329004E54502054494D454F55542832
:101290004E6F3429004E545020494C4C4547414C28
:1012A000205245502E004E5450204C454150204174
:1012B000444A5553540054494D4520494C4C4547E8
:1012C000414C0047505320464F524D415420455207
:1012D000524F52004E4D45412043484B53554D20EF
:1012E0004552522E0054494D45204441544120520C
:1012F000435645525200554E53594E432054494D82
:1013000045555000A010B110BA10C910D910E810FE
:10131000F6100611151123113111421153116011EC
:101320006C11791188119611A711B811C911DA1130
:10133000EB11FC110D121E122F12401251126212EB
:10134000731284129512A612B612C312D412E512A9
:10135000F6122D2D2F2D2D202D2D3A2D2D3A2D2D00
:1013600000484F55522020204D494E2E002A2A3A3F
:101370002A2A3A2A2A002D2D3A2D2D3A2D2D0054B5
:10138000494D450D0A00444154450D0A0061646A07
:1013900075737465640076616C69640053545553C9
:1013A0000D0A00444353540D0A005A444100524D63
:1013B0004300504645432C475074707300504D54C1
:1013C0004B3030312C3331342C330024504D544BBE
:1013D0003331342C302C312C302C312C302C302C1F
:1013E000302C302C302C302C302C302C302C302C1D
:1013F000302C302C302C312C302A32390D0A00247C
:10140000504D544B3331342C302C312C302C312C6A
:10141000302C302C302C302C302C302C302C302CEC
:10142000302C302C302C302C302C302C302A3238D0
:101430000D0A004649582049502041444452455322
:101440005300464958205355424E4554204D415370
:101450004B004649582044464C5420474154455778
:1014600041590046495820444E5320534552564551
:10147000520044484350205553452F554E5553452F
:1014800000424C4F41444341535420414444522E66
:1014900000424C4F41444341535420494E54564C12
:1014A0000042434153542043414C20524543562E61
:1014B0000054494D45205A4F4E4500475053204E49
:1014C0004F444154412054494D4552004750532008
:1014D000554E53594E432054494D4552004E4D45AB
:1014E000412053454E54454E5345003150505320F2
:1014F000494E5055542045444745004E54502052C3
:10150000582054494D454F55540041444A55535471
:1015100020574944544800475053204241554420E5
:101520005241544500484F55522053595354454D4C
:10153000005155495420544F204D41494E00331419
:10154000421452146314721481149114A114B1142E
:10155000BB14CC14DD14EB14FB140A151715251558
:1015600031154A5354285554432B393A3030290009
:101570004B5354285554432B393A303029004343B8
:1015800054285554432B383A3030290055544328B9
:1015900055544320303A3030290050535428555484
:1015A000432D383A30302900484454285554432DAF
:1015B000393A30302900621570157E158C159A1550
:1015C000A815907E0000907E000080700000000052
:1015D0000000808FFFFF7081FFFF465552554E4F30
:1015E000282447507470732900554E49562E2824DC
:1015F0004750524D432900554E49562E28244750F6
:101600005A44412900DA15E915F71546414C4C209A
:101610004544474500524953452045444745000B42
:1016200016151644495341424C4500454E41424C23
:10163000450023162B1644495341424C4500454E64
:1016400041424C45284E5450204D4F4445290036C8
:10165000163E162031323030627073002032343042
:10166000306270730020343830306270730020397B
:10167000363030627073003139323030627073004E
:101680003338343030627073003537363030627042
:10169000730053165C1665166E167716801689163B
:1016A000323420484F55522053595354454D00323F
:1016B0003820484F55522053595354454D0033302C
:1016C00020484F55522053595354454D00A016AF52
:1016D00016BE1657494454483A20202020207365EE
:1016E000630054494D454F55543A20202020206D29
:1016F0007300544F55543A20202020207365630016
:10170000544F55543A202020202073656300494EE1
:1017100054455256414C3A202020202073002F314E
:1017200038002D2D204D454E55202D2D0000112423
:101730001FBECFEFD0E1DEBFCDBF12E0A0E0B1E031
:10174000E4E3F9EC02C005900D92A43DB107D9F78E
:101750001CE0A4EDB2E001C01D92AD33B107E1F78A
:101760000E94060F0C9498640C94000080919201E2
:10177000882359F48091020A9091030A9093200CD7
:1017800080931F0C81E0809392010895A0E2B0E065
:10179000ECECFBE00C942D630E948A1A82E00E941C
:1017A0007E4C01C0A895F999FDCF86E090E065E0F8
:1017B00070E00E94936401C0A895F999FDCF8EE076
:1017C00090E060E570E00E94936401C0A895F999EB
:1017D000FDCF8CE090E06AE070E80E94936401C065
:1017E000A895F999FDCF80E290E044E651E068EADF
:1017F00070EC0E948B6401C0A895F999FDCF84E23A
:1018000090E040E05FEF6FEF7FEF0E948B6401C0DC
:10181000A895F999FDCF88E290E041E051E068EAAF
:1018200070EC0E948B6401C0A895F999FDCF8CE201
:1018300090E041E051E068EA70EC0E948B64CE01D8
:10184000019668EF70E00E94866301C0A895F9993F
:10185000FDCFCE01019660E170E040E150E00E94D2
:10186000736401C0A895F999FDCF8E010F5F1F4FDA
:10187000C80168E071E00E948663C80160E470E01E
:1018800040E250E00E94736401C0A895F999FDCF31
:101890008E010F5F1F4FC8016CE171E00E948663EB
:1018A000C80160E670E040E250E00E94736401C04D
:1018B000A895F999FDCF8E010F5F1F4FC8016CE20B
:1018C00071E00E948663C80160E870E040E250E089
:1018D0000E94736401C0A895F999FDCF8E010F5F36
:1018E0001F4FC8016CE371E00E948663C80160EA83
:1018F00070E040E250E00E94736401C0A895F9993D
:10190000FDCF80EC90E04FEF51E068EA70EC0E9470
:101910008B6401C0A895F999FDCF84EC90E060E05C
:1019200070E00E94936401C0A895F999FDCF86EC00
:1019300090E060ED77E00E94936401C0A895F9996A
:10194000FDCF88EC90E068E873E10E94936401C0E9
:10195000A895F999FDCF8CE390E061E070E00E94DA
:10196000936401C0A895F999FDCF8CEC90E060E0FC
:1019700070E00E94936401C0A895F999FDCF80EDB5
:1019800090E064EB70E00E94936401C0A895F9991F
:10199000FDCF82ED90E064E873E00E94936401C0A3
:1019A000A895F999FDCF8EE390E065EA73EC0E946B
:1019B0009364A096E4E00C9449630F931F930E94F4
:1019C000EF1D83B180958F70873069F40E94C60B3C
:1019D0000E948A1A83E00E947E4C82E00E94714C31
:1019E000A895FECFA895F999FDCF8EE390E00E94CF
:1019F0003964855A934C21F00E94C60B01C0A8950A
:101A0000F999FDCF86E090E00E9439649C018150F5
:101A10008E3F08F025E02093A70401C0A895F9990E
:101A2000FDCF8EE090E00E94396490937F05809313
:101A30007E0501978E5F9F4F40F080E590E0909388
:101A40007F0580937E0501C0A895F999FDCF8CE0B4
:101A500090E00E9439649C019F7790936E08809378
:101A60006D08C90101978E5F9F4F50F084E180930C
:101A700070088CE390E090936E0880936D0810C01E
:101A800037FF0CC08091060A9091070A019711F068
:101A900084E101C085E18093700802C01092700853
:101AA00080917008882309F040C080E290E044E60D
:101AB00051E068EA70EC0E949E1C609345057093AB
:101AC0004605809347059093480584E290E040E006
:101AD0005FEF6FEF7FEF0E949E1C6093490570934C
:101AE0004A0580934B0590934C0588E290E041E0D5
:101AF00051E068EA70EC0E949E1C60934D05709363
:101B00004E0580934F05909350058CE290E041E0A4
:101B100051E068EA70EC0E949E1C6093F909709392
:101B2000FA098093FB099093FC0980E190E069EE4B
:101B300079E048EF50E00E947B1C8091030162EF46
:101B400079E00E94473C8091040164EF79E00E94B3
:101B5000473C8091050166EF79E00E94473C80EDAB
:101B600090E00E9439642FEF8F3F920711F484EBCD
:101B700090E09093010A8093000A82ED90E00E9429
:101B800039644FEF8F3F940711F484E893E090930A
:101B9000030A8093020A80E490E06CE877E048E072
:101BA00051E00E94581C80E690E06CEA77E04CE13E
:101BB00051E00E94581C80E890E06CEC77E04CE229
:101BC00051E00E94581C80EA90E06CEE77E04CE314
:101BD00051E00E94581C80EC90E04FEF51E068EA21
:101BE00070EC0E949E1C60931208709313088093FF
:101BF00014089093150801C0A895F999FDCF84ECBD
:101C000090E00E94396490933308809332088F5F8C
:101C10009F4F31F4109233081092320801C0A895FA
:101C2000F999FDCF86EC90E00E94396490933108D9
:101C30008093300801978E5F9F4F40F080ED97E0D2
:101C4000909331088093300801C0A895F999FDCF91
:101C500088EC90E00E9439649093380880933708AC
:101C60008F5F9F4F31F488E893E190933808809319
:101C700037081091FF09012F077011F011C0A895C6
:101C8000F999FDCF8AEC90E00E94396497FD08C075
:101C900080FF06C0187F11601093FF0901C0A8954E
:101CA000F999FDCF8CE390E00E9439649C014FEFDD
:101CB0008F3F940711F420E030E00230E1F480918E
:101CC000FF09877C8093FF09622F70E0AB014770AA
:101CD00050704130510511F4886004C04230510504
:101CE00019F480618093FF0963FF05C08091FF09AB
:101CF00080648093FF09832F83708093180A01C04A
:101D0000A895F999FDCF8CEC90E00E9439648093FE
:101D10000D0A8F3F21F410920D0A01C0A895F99980
:101D2000FDCF80910D0AE82FF0E0EE0FFF1FEE0FC0
:101D3000FF1FEE53FA4E85919591A591B491809332
:101D4000890190938A01A0938B01B0938C011F911C
:101D50000F910895EF92FF920F931F93E090320836
:101D6000F090330800E010E085E691E06DE171E06D
:101D70000E94743FE61AF70A080B190BB701C80155
:101D80001F910F91FF90EF900895EF92FF920F93A4
:101D90001F93E0903408F09035080027F7FC009579
:101DA000102F83E591E06DE171E00E94743FE61A27
:101DB000F70A080B190BB701C8011F910F91FF908B
:101DC000EF9008950F931F938C010E94663E00517F
:101DD00010406F717070060F171F10933508009335
:101DE00034080C33110534F48CE390E090933508FB
:101DF00080933408A3E5B1E0EDE1F1E082E10190E8
:101E00000D928150E1F71F910F910895AEE1B0E07E
:101E1000ECE0FFE00C941F63F894109268001CBA89
:101E20001DBA89E88093640080E885BF85BF80BFC4
:101E30009FEF92B980E185B918B813E01BB991B949
:101E400080EB84B98FE787B982EC8AB988E090E0AB
:101E50000E9433646093390870933A0880933B087A
:101E600090933C0889B18073803129F4119882E005
:101E70008093FF0905C0803239F412981093FF094E
:101E800089E08093930103C010981092FF0980E1CC
:101E90008CBD81E08DBD16BC92E094BD83E085BD14
:101EA00027EC27BD90936E001092B2009093B00083
:101EB00084E08093B1002093B3009093700084B7C6
:101EC00080FF04C081E00E94475013C081FF02C020
:101ED00082E007C082FF02C083E003C083FF09C025
:101EE00084E00E94475081E090E09093070A80933D
:101EF000060A14BE8CE028E130E00FB6F894A895ED
:101F0000209360000FBE8093600078940E94091BAC
:101F10000E94DD0C80E58CBD8091FF0987708230C6
:101F200011F58091A704882319F484E395E01FC07C
:101F3000813019F48AE992E01AC0823019F48CE4F5
:101F400091E015C0833089F0843019F482E590E087
:101F50000EC0853019F489E290E009C0863059F44A
:101F60008BE190E004C0833089F485EA90E090939F
:101F7000C5008093C40082E08093C00086E0809317
:101F8000C20088E98093C1008091C6005E9A80E11A
:101F900090E00E945C1B0E942D16882381F484E14E
:101FA00062EA7AE00E945C150E948A1A81E10E942E
:101FB0007E4C88E00E94714C1798A895FECF0E9435
:101FC00003190E948A1A80E00E947E4C80E00E94E1
:101FD000714C88E061E04CE750E00E94BB1A4090F1
:101FE000FF0927E042220E94631B8C010CC0A895C8
:101FF00032E0431619F40E94AB5305C083E0481643
:1020000011F40E94A4510E94631B801B910B805D00
:10201000974068F30E948A1AB3E04B1631F48EE0C1
:102020000E947E4C87E00E94714C8091FF0987FFDF
:102030000BC085E00E947E4C89E00E94714C80912B
:10204000FF0988730E943A53809170088823F1F049
:1020500081E090E09093720880937108A8E0B1E06D
:10206000EDE1F1E082E101900D928150E1F7809184
:102070007008843119F40E94C32803C086E10E94CD
:10208000A129882339F00E94475004C01092720899
:102090001092710822E0421649F48091FF0986FFF0
:1020A00002C083E007C04092690006C033E04316D7
:1020B00031F482E0809369001CBA81E08DBB1092FC
:1020C000070A1092060A0E94631B9E8F8D8FA895A7
:1020D0000E949C22823019F40E94082109C083309A
:1020E00019F40E947C2704C0843059F50E94E92429
:1020F000182F0E94B616112321F18091FF0990E05C
:1021000087709070892BD1F4163091F480910E0A6B
:102110008823A1F0A3E5B1E0EDE1F1E082E10190D7
:102120000D928150E1F71092E60910920E0A06C056
:102130001B3121F480E490E00E94E20E812F0E9486
:10214000475082E0481619F40E94AB5305C093E053
:10215000491611F40E94A451F89420901B0C309061
:102160001C0C10921C0C10921B0CA0911D0CB09119
:102170001E0CBC8FAB8F10921E0C10921D0C78940D
:10218000B1E02B16310431F02B8D3C8D213031051F
:1021900009F06CC2F89480918D0190918E01A0910C
:1021A0008F01B091900189839A83AB83BC8378942B
:1021B000CE0101960E94A21E009729F430EC3093C4
:1021C000060181E0B1C0AFE2B1E0FC0182E1019023
:1021D0000D928150E1F780910601803461F5809184
:1021E000270C8823F9F48091330190913401892BD5
:1021F000C9F48091310190913201892B99F4809139
:102200002F0190913001892B69F489819A81AB81EA
:10221000BC810197A109B10989839A83AB83BC83EF
:1022200082E043C08091270C823009F055C081E0E4
:102230008093270C51C0803809F04EC08091270C44
:10224000882309F049C08091330190913401479768
:1022500009F042C08091310190913201CB97E1F5B4
:1022600080912F0190913001CB97B1F589819A81AE
:10227000AB81BC810196A11DB11D89839A83AB837B
:10228000BC8380918D0190918E01A0918F01B091BE
:1022900090010196A11DB11D80938D0190938E0137
:1022A000A0938F01B093900181E08093270CCE0121
:1022B00001960E94A21EAFE2B1E0FC0122E1019072
:1022C0000D922150E1F7892B39F480EC80930601BF
:1022D00010921E0C10921D0C89819A81AB81BC81D9
:1022E0002091890130918A0140918B0150918C019C
:1022F000820F931FA41FB51F89839A83AB83BC836E
:10230000CE0101960E94A21EADE1B1E0FC0182E186
:1023100001900D928150E1F78091270C813039F4C2
:10232000109206011092270C809393010AC08091AD
:10233000270C823031F4ACE3B0E0B0931E01A093DF
:102340001D01B1E02B16310409F03CC10E94FB1EB7
:102350000E94CE300E94A42A8091320890913308C6
:10236000892B61F180910F0A9091100A0197E1F495
:102370000E94AA0E3B014C011616170618061906F4
:102380004CF10E94B133882311F00E944750A5E61A
:10239000B1E0EDE1F1E082E101900D928150E1F7D1
:1023A00082E00E94DE5016C0A5E6B1E0EDE1F1E06A
:1023B00082E101900D928150E1F709C0A5E6B1E0FC
:1023C000EDE1F1E082E101900D928150E1F76624A8
:1023D000772443015090FF0927E0522280910E0A92
:1023E000882361F55520B1F40E94C50E5B016C0194
:1023F000161617061806190624F1809145059091C6
:102400004605A0914705B09148050097A105B10583
:10241000C1F010C033E0531689F48091290C882351
:1024200069F40E94C50E5B016C01161617061806AA
:1024300019063CF081E080930E0A03C0AA24BB2455
:10244000650180910C0A8F5F80930C0A8C33A9F48C
:1024500010920C0A8091080A9091090AA0910A0A28
:10246000B0910B0A0196A11DB11D8093080A9093AB
:10247000090AA0930A0AB0930B0A20918D013091AA
:102480008E0140918F01509190018091890190912E
:102490008A01A0918B01B0918C01280F391F4A1F2E
:1024A0005B1F29833A834B835C838091180A8130B8
:1024B00061F420543843404050402D833E834F8385
:1024C000588754E0E52EF12C10C0823019F0EE242C
:1024D000FF240BC020563445404050402D833E839E
:1024E0004F83588746E0E42EF12CCE0105960E94DA
:1024F000A21EDE011996FC0182E101900D9281502D
:10250000E1F70F851889CE0101960E94A21EFC01F9
:10251000E114F104D1F08681978108171907A9F019
:10252000188B0F879F01AE01475F5F4F82E1DA0191
:102530000D90AD01D9010D929D018150C1F78481AB
:1025400095818E0D9F1D95838483A1E4B1E082E186
:1025500001900D928150E1F78091FD09882319F4D3
:102560000E946B4E2FC0843019F40E94474D2AC040
:10257000853021F5B2E05B1641F021E0521629F0DA
:1025800080910E0A882309F4EAC180E00E946A4C17
:102590008091320890913308892B61F080910F0A65
:1025A0009091100A019731F481E0B401A3010E94D7
:1025B000FD4C08C081E00E946A4C04C0863011F4D2
:1025C0000E948B4C8B8D9C8D019709F04FC08091A0
:1025D000FF09877029F410929301109292010BC0A9
:1025E000833049F0813069F50E94DE5010929301EA
:1025F0001092920126C08091340890913508209164
:10260000170A213019F4959587950BC0223049F4AB
:10261000880F991FA4E081309A071CF080E094E0B5
:1026200005C08034910514F480E490E00E94E20E2D
:10263000A3E5B1E0EDE1F1E082E101900D9281507E
:10264000E1F710920E0A80911B0190911C010197F5
:1026500069F410921C0110921B01A5E6B1E0EDE1B6
:10266000F1E082E101900D928150E1F78091E6095D
:102670008823D9F00E941F31182F8823E1F0805160
:102680008B3058F4A3E5B1E0EDE1F1E082E1019097
:102690000D928150E1F70E9470321092E60910927B
:1026A0000E0A812F0E94475006C01092E509109231
:1026B000E8091092E7098091FF098770823080F461
:1026C0000E940A33182F882359F01092E6091092BD
:1026D0000E0A80E490E00E94E20E812F0E94475093
:1026E000B1E02B163104F1F480915A05882359F09A
:1026F00080916B05815080936B05882321F480E0E5
:1027000090E00E94AB2480916C05882359F0809161
:102710007D05815080937D05882321F481E090E040
:102720000E94AB248091040A9091050A019711F44C
:102730000E94464F1092050A1092040A0E94631BE1
:102740002D8D3E8D821B930B409708F4A5C00E94EF
:10275000631B9E8F8D8F0E94E51B0E94F41B8823B4
:1027600009F49AC0179A9091FD09843141F480913F
:10277000FE09882309F090C00E947B5A5AC081311B
:1027800049F49F5F80911A01891708F0EEC090917B
:10279000FE09EBC0823149F48091FE09981719F4C3
:1027A00090911A01E2C09150E0C08331D1F4809140
:1027B000FE09882339F487E08093FE0996E190931F
:1027C0001A012AC0873039F4A7E1A093FE09B6E2C6
:1027D000B0931A0128C01092FE0926E020931A0136
:1027E0002DC0863189F480910F0A9091100A0197CB
:1027F00009F052C00E94B133882311F00E94475063
:1028000082E00E94DE5048C0883179F48091FE0950
:10281000873021F40E94315097E0A7C0873109F03A
:10282000A4C00E943C5097E1A0C08F3049F40E94A0
:10283000091B1092FE0936E030931A0190E095C012
:10284000803151F58091FF098770823088F4809142
:102850000E0A882309F58091450590914605A091BF
:102860004705B09148050097A105B105A9F002C040
:10287000833091F481E080930E0A0EC0892F875037
:102880000E94874D09C0873129F4892F87510E9402
:10289000F84D02C00E94464F80919201882321F09A
:1028A00080919201813099F481E090E09093100A38
:1028B00080930F0A8091FF0987708250823028F43C
:1028C0001092060181E08093070115981EC0809147
:1028D0009201833029F484E08093920185E208C05C
:1028E00080919201823031F494E09093920186E2DB
:1028F0000E9447501092100A10920F0AA0ECA09369
:102900000601B0E1B0930701159A809132089091C9
:102910003308892B41F080910F0A9091100A01979A
:1029200011F4149801C0149A80917008882371F0F2
:102930008091450590914605A0914705B0914805C5
:102940000097A105B10511F0139801C0139A0E94D8
:102950006616813011F41698BACB169AB8CB80E07F
:10296000B601A5010E94FD4C13CE9093FD09809104
:10297000FE09873009F087CF81CF8EBD0DB407FEE9
:10298000FDCF08952C988EBD0DB407FEFDCF1EBC63
:102990000DB407FEFDCF8EB52C9A08952C988EBDF0
:1029A0000DB407FEFDCF1EBC0DB407FEFDCF8EB5E6
:1029B0001EBC0DB407FEFDCF8EB52C9A08952C9841
:1029C000805C8EBD0DB407FEFDCF6EBD0DB407FE5D
:1029D000FDCF2C9A08950F931F93182F0E94C214B5
:1029E000082F812F8F5F0E94C214982F802F1F9174
:1029F0000F9108950F931F93182F0E94CE14082F44
:102A0000812F8F5F0E94CE14982F802F1F910F91DE
:102A100008950F931F93182F072F0E94DF14812F03
:102A20008F5F602F0E94DF141F910F9108952C98E3
:102A300080588EBD0DB407FEFDCF6EBD0DB407FEF0
:102A4000FDCF2C9A08952C9880568EBD0DB407FEAC
:102A5000FDCF6EBD0DB407FEFDCF2C9A08951F93D8
:102A6000182F8FE163E00E9423158FE1612F0E94F0
:102A700017151F9108951F93182F82E00E942F159C
:102A800084E1612F0E94DF1482E161E00E94DF1483
:102A900083E00E942F158AE00E94CE1480FDFBCFB8
:102AA00082E00E942F1582E160E00E94DF1488E13D
:102AB0000E94FA141F910895FF920F931F93F82E0E
:102AC0008B0182E00E942F1584E16F2D0E94DF149C
:102AD00086E1B8010E94091583E00E942F158AE063
:102AE0000E94CE1480FDFBCF1F910F91FF9008959F
:102AF0002C988AE38EBD0DB407FEFDCF1EBC0DB42D
:102B000007FEFDCF8EB52C9A08952C988AE38EBDD2
:102B10000DB407FEFDCF1EBC0DB407FEFDCF9EB564
:102B20001EBC0DB407FEFDCF8EB52C9A08952C98CF
:102B30008AE38EBD0DB407FEFDCF1EBC0DB407FEAB
:102B4000FDCF9EB51EBC0DB407FEFDCF8EB51EBCDD
:102B50000DB407FEFDCF7EB51EBC0DB407FEFDCF44
:102B60006EB52C9A0895FC012C988AE38EBD0DB4A5
:102B700007FEFDCF20E030E008C01EBC0DB407FE0C
:102B8000FDCF8EB581932F5F3F4F26173707A8F3F0
:102B90002C9A0895982F2C988AE78EBD0DB407FEC5
:102BA000FDCF9EBD0DB407FEFDCF2C9A0895282FB2
:102BB0002C988AE78EBD0DB407FEFDCF9EBD0DB4E7
:102BC00007FEFDCF2EBD0DB407FEFDCF2C9A089554
:102BD000282F2C988AE78EBD0DB407FEFDCF9EBD31
:102BE0000DB407FEFDCF2EBD0DB407FEFDCF7EBD9B
:102BF0000DB407FEFDCF6EBD0DB407FEFDCF2C9AC0
:102C00000895FC012C988AE78EBD0DB407FEFDCF18
:102C100020E030E008C080818EBD0DB407FEFDCFFE
:102C20002F5F3F4F319626173707A8F32C9ACB0119
:102C30000895282F2C988AE78EBD0DB407FEFDCF8E
:102C400080E090E005C02EBD0DB407FEFDCF0196DB
:102C500086179707C0F32C9A08958FE160E00E94D1
:102C6000DF1480E160E070E00E94091582E16FEFFF
:102C70007FE10E9409158AE06FEF7FE10E9409154C
:102C800083E00E942F1587E067E00E94DF1487E051
:102C90000E94C21480FDFBCF87E062E00E942315F2
:102CA0008FE160E30E9417158FE10E94C21485FD39
:102CB000FBCF80E00E942F1586E10E94EB1420E0FC
:102CC0008750984F09F421E0822F089581E00E94F7
:102CD0003B159695879596958795817008958FE118
:102CE0000E94C2148095881F8827881F0895EF923C
:102CF000FF920F931F938C0180E00E942F1580E0BC
:102D00000E94FA14F82EE92E6091AF047091B0047D
:102D10006A5F7F4F600F711F89E1683D780710F08F
:102D2000685D794180E00E9409158F2D9E2D1F91CD
:102D30000F91FF90EF900895EF92FF920F931F93E2
:102D40008C0180E00E942F1582E00E94FA14F82E78
:102D5000E92E0752164E82E0B8010E9409158F2D08
:102D60009E2D1F910F91FF90EF9008950F931F9349
:102D70000091B1041091B2040150104080E00E9413
:102D80002F158EE160E40E941715B80189E1083D16
:102D9000180710F067ED79E18CE00E9409151F918A
:102DA0000F9108951F93CF93DF9381E00E942F1519
:102DB00089E10E94C214182F80E00E942F158EE036
:102DC0000E94C214C82FD0E081E00E942F1589E133
:102DD0000E94C214181779F78CE00E94EB149F71BF
:102DE0008C179D0720F49C012952364E09C0C81744
:102DF000D90719F427ED39E105C09C012150304075
:102E00002C1B3D0BC901DF91CF911F910895A7E0C5
:102E1000B0E0EDE0F7E10C9427638C01E090B4049E
:102E2000F090B504E80EF91E82E0B8010E94091581
:102E300080E00E94CA1584E0B8010E94091586E06E
:102E4000B7010E9409158FE160E80E9417158FE114
:102E500060E80E9423158CE16AE00E9423158FE14F
:102E600068E00E9417158091B3048550823008F005
:102E700068C000E010E08CE10E94C2148A7031F456
:102E80000F5F1F4F83E0083E1807A9F78CE10E94EF
:102E9000C21481FD05C083E0083E180708F451C044
:102EA0008FE168E00E94231580E00E94FA145C0123
:102EB00086E00E94FA146C010894C11CD11C80E0C9
:102EC000B6010E9409158E010F5F1F4FC80167E010
:102ED00070E00E94B315EE24F02E012F8CE10E94C9
:102EE000C21481FF2AC08C8185FF27C08FE160E872
:102EF0000E9417158FE160E80E9423158CE16AE0BB
:102F00000E9423158FE168E00E9417158CE10E9452
:102F1000C2148A70D9F38FE168E00E94231580E023
:102F2000B6010E9409158F2D902F67E070E00E9476
:102F3000B315E39480E1E81689F680E0B5010E94BC
:102F400009152796EAE00C944363A0E0B0E0EBEAB1
:102F5000F7E10C942863B82E282F392F6901EE244D
:102F6000FF24870111C00E947815D82F0E94781580
:102F7000C82FCE01A0E0B0E0E80EF91E0A1F1B1F0B
:102F80008EEF9FEFC80ED91E92E0C916D10458F7F4
:102F9000C701D8019C01AD01B0FE0BC00E9478159D
:102FA000D82FC0E09E0140E050E02E0D3F1D401F95
:102FB000511F203080E0380781E0480780E0580743
:102FC000A0F0CA0140E050E0A0E0B0E0280F391FB7
:102FD0004A1F5B1F203090E0390791E0490790E0DD
:102FE000590718F0C90101969C01C901CDB7DEB798
:102FF000E9E00C9444630F931F938B010E947716B2
:10300000C8010E94A5179C0120953095C9011F9108
:103010000F910895EF92FF920F931F938C017B0104
:1030200080E00E942F150752164E80E0B8010E94E2
:103030000915C7010E94A5179C0120953095C9016B
:103040001F910F91FF90EF900895A0E0B0E0EBE2A8
:10305000F8E10C9429636C017B018A01411551054B
:1030600009F444C04130510551F40E947716C7015C
:103070000E949C160E9478150E94CA1537C080E0F5
:103080000E942F15C091AF04D091B0042696CC0DAC
:10309000DD1D89E1C83DD80710F0C85DD94180E148
:1030A000BE010E940915B801615070406C0F7D1F70
:1030B00099E1683D790710F0685D794182E10E94ED
:1030C000091589ED99E1E80EF91E84E1B7010E9426
:1030D00009158FE160E10E9423158FE160E20E94F3
:1030E00017158FE10E94C21485FDFBCFCDB7DEB767
:1030F000E8E00C9445638FE164E00E9423158DE1C4
:103100000E94C21482FDFBCF8FE10E94C21487FD92
:10311000FBCF8EE160E20E94171508951F93182FD0
:1031200083E00E942F1585E1612F0E94DF141F911B
:10313000089583E00E942F1585E10E94C21408952E
:10314000FC012C988AE38EBD0DB407FEFDCF20E074
:1031500030E00AC01EBC0DB407FEFDCF8EB58193D2
:103160002F5F3F4F841719F02617370798F3108207
:103170002C9AC90108950F931F93CF93DF938C016D
:10318000C0E0D0E003C00E9478152196C017D10797
:10319000D0F3DF91CF911F910F910895CF93DF93DB
:1031A000EC010E948D63AC012C988AE78EBD0DB4B2
:1031B00007FEFDCF20E030E00AC0FE01E20FF31F62
:1031C000E491EEBD0DB407FEFDCF2F5F3F4F2417F6
:1031D000350798F32C9ACA01DF91CF9108958EE1BB
:1031E00060E20E94231580E190E00E945C1B8DE16B
:1031F0000E94C21483FDFBCF80FFF9CF8FE164E012
:103200000E94171508951F938EE160E20E94231516
:1032100080E190E00E945C1B5E9880E190E00E945B
:103220005C1B5E9A80E190E00E945C1B1FEF2C9873
:103230001EBD0DB407FEFDCF2C9A80E190E00E94E8
:103240005C1B8DE10E94C21483FDF1CF80FFEFCFA4
:103250008FE160EC0E94DF148EE160E80E94DF14D1
:1032600088E060E070E00E9409158CE067ED79E18C
:103270000E9409158AE067ED79E10E94091584E052
:1032800068ED79E10E94091581E00E942F1588E11F
:1032900061EA0E94DF1482E00E942F1580E06DE059
:1032A0000E94DF1481E060E00E94DF1482E062E3AC
:1032B0000E94DF148AE06EEE75E00E94091586E038
:1032C00062E17CE00E94091584E062E10E94DF1463
:1032D00083E060E40E94DF1489E06FE30E94DF1462
:1032E00083E00E942F1585E160E00E94DF1484E0F6
:1032F000609100010E94DF1485E0609101010E944D
:10330000DF1482E0609102010E94DF1483E060918B
:1033100003010E94DF1480E0609104010E94DF1429
:1033200081E0609105010E94DF1482E10E94C214D5
:103330008F718093B30480E060E070E00E945C15C0
:1033400080E160E071E00E945C1584E162E774E076
:103350000E945C1580E00E942F158FE164E00E94BE
:10336000DF141F910895CF93DF93EC0181E00E9459
:103370002F1589E10E94C214882321F40E942F1581
:1033800080E044C080E00E942F156091B1047091EC
:10339000B20480E00E9409158091B1049091B204BA
:1033A0009093B0048093AF0489EA94E066E070E003
:1033B0000E94B3158091AA048F718093AA04809112
:1033C000AC048F718093AC042091A9043091AA04BD
:1033D0003093B2042093B1048091AB049091AC047B
:1033E0008F5E954080F489E1283D380760F420FD28
:1033F0000AC08091AE0487FD06C08091AD0484FDB3
:1034000002C087FD06C00E94031982E0DF91CF91C0
:103410000895F89480918D0190918E01A0918F0173
:10342000B09190018093220890932308A0932408E0
:10343000B09325088091190C90911A0C90932B0849
:1034400080932A087894CE016EE070E00E94B31554
:1034500081E0DCCF98B18F70907F892B88B9089577
:10346000469898B18F70907F892B88B90000449A54
:1034700083E090E00E945C1B449808951F93182FEE
:1034800088B1912F92959F70807F982B98B9449A1C
:1034900083E090E00E945C1B449888B11F70807F9D
:1034A000812B88B9449A83E090E00E945C1B449889
:1034B0001F910895469A0E943E1A089546980E94C8
:1034C0003E1A08950E945A1A81E090E00E945C1B07
:1034D0000895CF93DF93EC0103C021960E94621AF6
:1034E00088818823D1F7DF91CF91089580E10E94F0
:1034F0005E1A81E090E00E945C1B0895882311F41D
:103500008CE001C08EE00E945E1A81E090E00E9493
:103510005C1B089581E00E945E1A89E190E00E94A0
:103520005C1B0895662349F0613011F4805C05C08E
:10353000623011F48C5E01C08C5A80680E945E1A61
:1035400081E090E00E945C1B08950F931F93042F6D
:103550000E94921A10E004C080E20E94621A1F5F6B
:103560001017D4F31F910F910895682F80E040E168
:103570000E94A51A0895CF93DF93EA010E94921A40
:1035800003C00E94621A2196FE0184918823C9F724
:10359000DF91CF9108950F931F938A010E94921A91
:1035A000C8010E94691A1F910F9108951F93142F4B
:1035B0000E94921A812F0E945A1A81E090E00E9484
:1035C0005C1B1F9108950F931F93CF93DF938B0183
:1035D000880F880F880F887380640E945E1AC0E08D
:1035E000D0E081E090E00E945C1B81E090E00E94CE
:1035F0005C1BF801EC0FFD1FE4918E2F0E945A1AFC
:103600002196C830D10569F7DF91CF911F910F91B5
:1036100008951F93CF93DF9388E290E00E946B1B85
:1036200083E00E94301A82E490E00E945C1B83E0F9
:103630000E94301A81E090E00E945C1B83E00E94AF
:10364000301A81E090E00E945C1B82E00E94301AF8
:1036500081E090E00E945C1B88E20E945E1A81E09B
:1036600090E00E945C1B88E00E945E1A81E090E07E
:103670000E945C1B81E00E945E1A89E190E00E943A
:103680005C1B86E00E945E1A81E090E00E945C1B59
:103690008CE00E945E1AC4ECD0E010E0FE0165915F
:1036A0007491812F0E94E31A1F5F22961830B1F7A0
:1036B000DF91CF911F91089528EC00002A95E9F73A
:1036C0000197D1F70895F8942091D4023091D50252
:1036D0007894C9010895AC01F8942091D4023091F6
:1036E000D502789401C0A895F8948091D402909165
:1036F000D5027894821B930B84179507A0F3089545
:10370000DC01F8947894809121048823A1F0F89446
:10371000E0911F04F0E0E15EFC4F80818C9380918A
:103720001F048F5F80931F04809121048150809338
:103730002104789481E00895A1E0B0E0E2EAFBE1A1
:103740000C942D638E010F5F1F4F01C0A895C80117
:103750000E94801B8130D1F32196E4E00C944963F0
:10376000A1E0B0E0E6EBFBE10C942F63CE01019603
:103770000E94801B882321F19091A2049F3740F082
:103780001092A6041092A5041092A20482E019C01F
:103790008981E92FF0E0EE5DFB4F8083E92FEF5F39
:1037A000E093A2048A3061F4F0E0EE5DFB4F1082FA
:1037B0001092A2041092A6041092A50481E001C008
:1037C00080E02196E2E00C944B639091DA0283B1A1
:1037D000E6EDF2E0E90FF11D80958F7080839F5F29
:1037E00093709093DA0208959091D7028091D60257
:1037F00098238091D80298238091D902982341F18F
:10380000983011F494E11DC0943011F493E119C083
:10381000923011F492E115C0913011F491E111C090
:103820009C3011F498E10DC0933011F49FE009C071
:10383000993011F490E105C09A3011F090E001C088
:1038400096E180912A0C981729F090932A0C03C0D6
:1038500010922A0C90E0892F0895EF92FF920F9317
:103860001F93CF93DF93F894E090D402F090D502A9
:1038700078948701A895F894C091D402D091D5028C
:103880007894CE01801B910B409718F00E94E51BA5
:103890008E010E94F41B882331F4CE19DF09C05138
:1038A000D74240F389E1CDB7DEB7E6E00C94476339
:1038B0000F931F93CF93DF939C01EB018A0101C00B
:1038C000A895F999FDCFCE01B9014FE150E00E94D2
:1038D00023641F8E8881992787FD90950E945663E7
:1038E000892B21F4CE01B8010E948663DF91CF912C
:1038F0001F910F9108950F931F93CF93DF939C0116
:10390000EB018A0101C0A895F999FDCFCE01B9015B
:103910004FE050E00E9423641F868881992787FD2D
:1039200090950E945663892B21F4CE01B8010E9424
:103930008663DF91CF911F910F910895EF92FF92CF
:103940000F931F93142F052FF62EE72E01C0A89575
:10395000F999FDCF0E9433649B01AC012F3F8FEF9B
:1039600038078FEF48078FEF580741F4212F302F8A
:103970004F2D5E2DC901DA019C01AD01B901CA01CB
:103980001F910F91FF90EF9008951F93CF93DF93B6
:10399000EC010E948D63182F813414F580911D0372
:1039A00090911E03019711F4A895FECF81E090E05D
:1039B00090931E0380931D038BED92E0BE010E9445
:1039C00086638091DB028093C600115010931C0324
:1039D00081E080931B038091C10080668093C100C9
:1039E000DF91CF911F9108951F93BC01FC010190BD
:1039F0000020E9F731971E2F181B11340CF5809128
:103A00001D0390911E03019711F4A895FECF81E04C
:103A100090E090931E0380931D038BED92E00E9433
:103A2000FF638091DB028093C600115010931C034A
:103A300081E080931B038091C10080668093C10068
:103A40001F9108951F93482F792F162F613444F545
:103A500080911D0390911E03019711F4A895FECF4C
:103A600081E090E090931E0380931D032BED32E0E4
:103A7000E62FFF27E7FDF095C901642FAF010E94F3
:103A8000BE638091DB028093C600115010931C032B
:103A900081E080931B038091C10080668093C10008
:103AA0001F9108950000000008952D9A2F9800009E
:103AB00000002F9A90E087FF02C02D9A01C02D9838
:103AC0002F98000000002F9A9F5F983011F0880F08
:103AD000F2CF08951F93CF93DF93182FEB018091BE
:103AE000A804813021F4CB010E94D73EEC01F89468
:103AF0002F9A5F9A80E30E94551D5F982F9A5F9AD4
:103B00001F73812F80640E94551D80E0D7FF02C083
:103B10002D9A01C02D982F98000000002F9A0000C8
:103B200000008F5F803119F0CC0FDD1FEFCF5F9861
:103B30002D985F9A000000001E9BFECF5F985F9853
:103B40007894DF91CF911F9108951F93CF93DF93C6
:103B5000C0E0D1E012E0688179812296812F0E9435
:103B60006A1D1F5F1530B9F7DF91CF911F9108953E
:103B7000FF920F931F93182F062FF72EBA010E9462
:103B80006A1D812F8F5F602F7F2D0E946A1D1F91FC
:103B90000F91FF900895F8942F9A5F9A8F73806821
:103BA0000E94551D80E020E030E02F9800000000CA
:103BB0002F9A00000000220F331F1E9921608F5F93
:103BC000803199F7932F5F9878948091A804813081
:103BD00021F4822F0E94D73E9C01C90108951F93B2
:103BE000CF93DF9380E00E94CB1D8050904419F466
:103BF00081E08093A80482E00E94CB1D8F5F9F4FDD
:103C000061F012E0C0E0D1E0812F0E94CB1D8883DB
:103C1000998322961F5F1530B9F7DF91CF911F91DD
:103C200008959F92AF92BF92CF92DF92EF92FF9250
:103C30000F931F93182F042FB52EA62E972E0E9498
:103C4000CB1D6C01812F8F5F0E94CB1D7C018FEFFC
:103C5000C8168FEFD8068FEFE8068FEFF80641F40D
:103C6000202F3B2D4A2D592DC901DA016C017D0110
:103C7000B601C7011F910F91FF90EF90DF90CF9099
:103C8000BF90AF909F9008951F1D1F1E1F1E1F1FE6
:103C90001E1F1E1FCF93DF93EC012C964AE834D0F1
:103CA0006627772736E4AEE6B1E0532F537009F06C
:103CB0001197321729F078F56A0F7B1F3395F3CFF0
:103CC0004CE022D0E8E8FCE330E0C8953196313092
:103CD00011F451110A94321720F4600D711D3395BF
:103CE000F4CF402D439510D02150A8F0620F711DE4
:103CF0008827992748E108D015D04CE305D012D089
:103D00002CE302D00FD00BC03A912A912417310531
:103D100040F00F900F906FEF7FEF8FEF9FEFDF91ED
:103D2000CF91089551E2AA1B08F4A40FA795979587
:103D30008795779567955A95B9F7620F711D811D23
:103D4000911D0895CF93DF93FC0120813181428141
:103D50005381CC27DD2757FD3CC0CBE2DCE06CE390
:103D60003CD00882198239D00A821B8268E135D0A2
:103D70000C821D82F9012C5F3F4F67E02ED00C862C
:103D80001D869F01A6E4EEE6F1E0BA2FB37009F0BC
:103D900031972E173F0720F02E1B3F0BA395F3CF33
:103DA000AA871B862E873F87E8E8FCE3AA27C895E9
:103DB0003196A13011F4B1110A942015310520F08B
:103DC00020193109A395F3CFA887198623952E834F
:103DD0003F83CE01DF91CF910895002470E2220F3E
:103DE000331F441F551F001C061610F0061A23959A
:103DF0007A95A9F70895E6EEF4E08281813041F4E6
:103E000080819181019791838083892B09F41282AB
:103E10003D9685E0EE34F80781F70895CF92DF9262
:103E2000EF92FF920F931F936B017C018AE290E067
:103E30009093B5048093B40480E00E942F1582E033
:103E40006DEC7FE10E9409158FEF66E070E00E9443
:103E5000191600E011E0C80166E070E00E9401164A
:103E600086E098E00E94D71581E090E00E94D71587
:103E700080E098E00E94D71586E00E94CA1584E091
:103E80000E94CA1581E090E00E94D715C80166E043
:103E900070E00E9401166091450570914605809181
:103EA0004705909148050E94E81580E066E070E0C3
:103EB0000E941916C701B6010E94E8158CEC9FE11B
:103EC0000E9407171F910F91FF90EF90DF90CF9006
:103ED0000895EF92FF920F931F93CF93DF937B018F
:103EE0008C01E901ECEDF4E020E080819181A28178
:103EF000B3818E159F05A007B10711F4922F0DC055
:103F00002F5F3D96283089F7CD2BF9F0909144052D
:103F1000892F8F5F8770809344058DE0989FF00113
:103F20001124E452FB4FEF012496DA0186E00D9054
:103F300009928150E1F7E082F1820283138380EBE2
:103F400094E09387828781E08487CDB7DEB7E6E08F
:103F50000C944763ACE1B0E0E0EBFFE10C94256327
:103F6000CE0101966CE170E00E94B3158F819885B7
:103F70000E94D73E4C016F85788989899A890E9471
:103F8000DB3E5B016C01698D7A8D8B8D9C8D0E946F
:103F9000DB3E7B018C0189819A810E94D73E01978B
:103FA00009F071C08B819C810E94D73E805098405F
:103FB00009F069C08091450590914605A09147059B
:103FC000B0914805E816F9060A071B0709F05BC01F
:103FD000CE01439660E071E046E050E00E94066446
:103FE000009709F050C0AE14BF04C006D10611F40A
:103FF00082E04AC08E01075F1F4FC601B501A801CC
:1040000021E030E00E94691F81E088169104D9F513
:104010008CE190E09093B5048093B4048EE090E03E
:104020000E949C1681E090E00E94D71580E098E005
:104030000E94D71586E00E94CA1584E00E94CA1526
:1040400082E090E00E94D71580E091E066E070E0A9
:104050000E940116609145057091460580914705C3
:10406000909148050E94E815C80166E070E00E9442
:104070000116CE010F9664E070E00E94011686E002
:1040800098E00E94B22080E06C96ECE00C944163D2
:10409000EF92FF920F931F93E090BC04F090BD0449
:1040A0000091BE041091BF042091490530914A054A
:1040B00040914B0550914C05DA01C9018E299F2989
:1040C000A02BB12B8F5F9F4FAF4FBF4F49F486EBB3
:1040D00094E06FEF70E046E050E00E94D96335C095
:1040E0008091450590914605A0914705B0914805FE
:1040F0008E259F25A027B12782239323A423B523B0
:104100000097A105B10511F421E009C0E0904D052B
:10411000F0904E0500914F051091500522E0ECED16
:10412000F4E08485813099F480819181A281B3810A
:104130008E159F05A007B10751F4A6EBB4E03496A5
:1041400086E001900D928150E1F720E005C03D9698
:1041500085E0E434F80729F7822F1F910F91FF9033
:10416000EF9008950F931F938C018091B404909168
:10417000B5040E969093B5048093B40480E090E06B
:104180000E949C1686EB94E066E070E00E940116A7
:1041900080E091E066E070E00E940116C8010E9494
:1041A000D71588ED99E10E9407171F910F91089587
:1041B000AEE0B0E0EEEDF0E20C942E63CE0101969D
:1041C0000E94B3198823F1F0A6EBB4E0FE01379604
:1041D00086E001900D928150E1F78D859E850E94C9
:1041E000D73E28E08030920711F411E00CC08650D1
:1041F000984031F40E94AA1F182F0E94B61603C0DF
:104200000E94B61610E0812F2E96E3E00C944A63CC
:10421000A8E0B0E0EEE0F1E20C942D6382E290E0E1
:104220000E947716CE01019668E070E00E94B315F7
:104230008981809354058A81809355056091B404E7
:104240007091B50482E290E00E94FB17892B81F007
:104250008AE390E00E9477160E94971560935605B6
:1042600070935705809358059093590587E057C080
:1042700080915405883031F16D817E818F819885E0
:104280000E94DB3E9B01AC0160935605709357057D
:10429000809358059093590580915405833019F403
:1042A0000E9403193BC08530C9F5809155058130C6
:1042B000A9F520934D0530934E0540934F0550933B
:1042C00050052CC04091B4045091B50482E290E0B6
:1042D00062E270E00E94251882E290E00E949C1643
:1042E00080E00E94CA1580E00E94CA1580E090E03C
:1042F0000E94D7156091B4047091B50482E290E0F9
:104300000E940A188C0184E290E00E949C16C80169
:104310000E94D71581E00E94ED2101C08AE0289615
:10432000E4E00C944963A0E0B0E0E9E9F1E20C9428
:104330002863B82EEB016A01E0EDF4E0EE24FF24DF
:104340008701308121813296C901A0E0B0E0E80EFA
:10435000F91E0A1F1B1F84E0EC3DF80791F781E06E
:10436000B81651F480E00E942F15C752D64E80E057
:10437000BE010E94091503C0CE010E947716C60136
:104380000E94A5179C0140E050E02E0D3F1D401FEC
:10439000511F203080E0380781E0480780E058074F
:1043A000A0F0CA0140E050E0A0E0B0E0280F391FC3
:1043B0004A1F5B1F203080E0380781E0480780E01B
:1043C000580718F0C90101969C0120953095C90144
:1043D000CDB7DEB7E9E00C944463ACE1B0E0E3EFC5
:1043E000F1E20C942D63182F8091B4049091B504E0
:1043F00044969093B5048093B4048EE090E00E94BC
:104400009C1680E095E40E94D7158091B4049091A9
:10441000B5040E94D71580915105909152050E94D4
:10442000D71580E090E40E94D71580E40E94CA1559
:10443000812F0E94CA1580E090E00E94D7156091FC
:1044400045057091460580914705909148050E9469
:10445000E8156091BC047091BD048091BE049091F8
:10446000BF040E94E8158EE090E064E170E00E94D5
:104470000A188C0188E190E00E949C16C8010E94F5
:10448000D7150E944820882309F443C0DE01119605
:10449000E4EBF4E09CE101900D929150E1F7823061
:1044A00049F460914D0570914E0580914F059091B2
:1044B000500508C06091BC047091BD048091BE0499
:1044C0009091BF040E940E1F0E94B6160E94631BAB
:1044D0008C01A8950E94D820882311F00E94B6165E
:1044E0000E944820882311F420E008C00E94631B2A
:1044F000801B910B8858934160F326E0A4EBB4E055
:10450000FE0131968CE101900D928150E1F722235A
:1045100029F480E098E00E94B22020E080915105CB
:104520009091520501969093520580935105822FE8
:104530006C96E4E00C944963A4E1B0E0E2EAF2E2B4
:104540000C942B630E94D820882309F4A1C08230E8
:1045500011F485E09DC08EE090E064E170E00E947F
:10456000FB17892B09F091C08EE090E00E9477162E
:10457000CE01019664E170E00E94B31569897A89E1
:104580008B899C890E94DB3E7B018C01209149052F
:1045900030914A0540914B0550914C058981682F17
:1045A00070E0CB01807F90708034910509F06DC080
:1045B0008091450590914605A0914705B091480529
:1045C000E816F9060A071B0799F02E293F29402B08
:1045D000512B2F5F3F4F4F4F5F4F51F08FEFE8163A
:1045E0008FEFF8068FEF08078FEF180709F04DC01F
:1045F0006F707070660F771F660F771F609353059B
:104600008B819C810E94D73E20915305821B91098A
:104610009093B5048093B4046D857E858F859889C9
:104620000E94DB3E6093BC047093BD048093BE0483
:104630009093BF04E092C004F092C1040093C204BE
:104640001093C30480915305853120F0845190E08C
:104650000E94BB186091BC047091BD048091BE049F
:104660009091BF0446EB54E020E030E00E94691FC7
:104670008A85813011F482E00BC0813111F483E02E
:1046800007C0863011F484E003C00E94B61680E0B3
:104690006496E6E00C944763A0E0B0E0E2E5F3E264
:1046A0000C942A63D82EEB017A0184E190E0E80EA5
:1046B000F91EF092B504E092B4048CEE9FEFE80E80
:1046C000F91E82E290E00E949C168D819E810E94DC
:1046D000D7158F8198850E94D71569857A858B8536
:1046E0009C850E94E8156D857E858F8598890E943E
:1046F000E81580E50E94CA158D2D8F730E94CA159A
:1047000084EB95E00E94D71560E070E080E090E0D7
:104710000E94E81560914505709146058091470516
:10472000909148050E94DB3E6093D0047093D104C1
:104730008093D2049093D30469817A818B819C8188
:104740000E94DB3E6093D4047093D5048093D6041A
:104750009093D7041092D80486E08093D904809176
:10476000B4049091B5040E94D73E9093DB048093EB
:10477000DA044091B4045091B50481E062E270E043
:104780000E9493218C0182E390E00E949C16C80154
:104790000E94D71586E00E94ED21682F882301F53D
:1047A0008D2D90E083709070892B41F089859A85DA
:1047B000AB85BC850196A11DB11D0EC0E114F104AD
:1047C00079F0970140E050E089859A85AB85BC85FA
:1047D000820F931FA41FB51F89879A87AB87BC8759
:1047E000862FCDB7DEB7E7E00C944663A2E1B0E0D8
:1047F000ECEFF3E20C942F632091C4043091C504D4
:10480000C901A0E0B0E08A839B83AC83BD83809123
:10481000C6049091C7049F838E83398728871A86A0
:104820001B861C861D868091CC049091CD04A0919E
:10483000CE04B091CF040196A11DB11D8E879F8734
:10484000A88BB98B84E0BE016F5F7F4F40E050E0E2
:104850000E944C236296E2E00C944B63A8E0B0E027
:10486000E4E3F4E20C9425637C018091C804909108
:10487000C9040E94771600E010E06E010894C11C84
:10488000D11C26E8A22E27E0B22EAE0CBF1C92E06F
:10489000892E9924939453C0C60165E070E04AE0E4
:1048A0000E94A018080F191FC60169ED70E00E9450
:1048B0007D63892B91F4E114F10419F082E896E00C
:1048C00002C082E895E06BEF70E04AE00E94A01819
:1048D000080F191FF501908232C0C60164ED70E027
:1048E00044E050E00E949663892B19F4F501808220
:1048F00026C089818D30E1F48A818A30C9F48091A3
:10490000CA049091CB0408171907C8F0EE0CFF1CDD
:1049100082E897E0E80EF91E81E090E0F7019183CC
:10492000808315C00F5F1F4F0E9478158A3039F0C1
:104930008091CA049091CB040817190798F38091CD
:10494000CA049091CB040817190708F4A5CF28963C
:10495000ECE00C944163CF93DF93EC01009719F0E6
:1049600022E836E002C022E835E0FE01EE0FFF1F2C
:10497000DF0143E0AA0FBB1F4A95E1F7AE0FBF1F4F
:10498000A65ABA4F1C9211961D921D921D921C920E
:10499000149716961C921E92159718961C921E92AA
:1049A00017971D961D921D921D921C92509780E0A4
:1049B00091E0D901AC011D9241505040E1F7EE5712
:1049C000F84F11821082CA57D84F1882DF91CF91C9
:1049D0000895A6E2B0E0EFEEF4E20C9421630091BA
:1049E000530510E0025F1F4FCE01439664E170E073
:1049F0000E94B3158B899C890E94D73E9093C50471
:104A00008093C4048D899E890E94D73E9093C704E9
:104A10008093C6046F89788D898D9A8D0E94DB3EC4
:104A20006093CC047093CD048093CE049093CF0414
:104A30002F8D2695269530E0C801820F931F909305
:104A4000C9048093C8048091B4049091B504821B7A
:104A5000930B9093CB048093CA046091BC04709133
:104A6000BD048091BE049091BF040E94DB3E609320
:104A7000D0047093D1048093D2049093D3046091B6
:104A8000C0047091C1048091C2049091C3040E943B
:104A9000DB3E6093D4047093D5048093D604909346
:104AA000D7041092D80486E08093D9048091B4048E
:104AB0009091B5040E94D73E9093DB048093DA0472
:104AC0004091B4045091B50480E0B8010E94932154
:104AD000892B09F099C198A1992309F495C1609097
:104AE000BC047090BD048090BE049090BF04E09020
:104AF000C404F090C504A090C604B090C7040AE5B1
:104B000015E0CC24DD246FEF7FEF2E010894411CCB
:104B1000511CD201F80182E101900D928150E1F720
:104B2000AE81BF81E885F9852A813B814C815D8119
:104B30008981882331F48FEF6F3F780711F4B60134
:104B40000BC0261537054805590531F4EE15FF054C
:104B500019F4AA15BB05C1F00894C11CD11C0E5E46
:104B60001F4FE2E0CE16D104A1F6FFEF6F3F7F07A3
:104B700041F06B01C094D0948CE9C8168FEFD80631
:104B800019F40E94F623FFC0D7FE47C091FF3FC132
:104B900080917E0590917F05A816B90609F037C16E
:104BA000C094D094C601880F991F8C0143E0000F78
:104BB000111F4A95E1F7080F191F065A1A4FF801FD
:104BC0006182728283829482B682A582F086E782B5
:104BD00081E080830E94663EF80161877287838747
:104BE00094878091CC049091CD04A091CE04B09193
:104BF000CF040196A11DB11D85879687A787B08B2D
:104C00008CE3818B82E1B80140E050E00E944C23AC
:104C1000F82E882309F4FCC053C091FF03C00E9402
:104C2000F6234DC092FF0FC0B601660F771FCB0170
:104C300023E0880F991F2A95E1F7680F791F665ABC
:104C40007A4F84E038C090FF3FC0C601880F991F9B
:104C50008C01B3E0000F111FBA95E1F7080F191F7F
:104C6000065A1A4FF80120818091CC049091CD040E
:104C7000A091CE04B091CF040196A11DB11D8587EE
:104C80009687A787B08B223079F480E1B80140E0A5
:104C900050E00E944C2381E1B80140E050E00E94C6
:104CA0004C23F82E85E0A1C0233019F0263009F0FE
:104CB000AEC080E1B80140E050E00E944C23F82EE5
:104CC000C6010E94AB24A4C093FF5FC08091CA04B8
:104CD0009091CB04009711F480E055C05601AA0CC6
:104CE000BB1C8501F3E0000F111FFA95E1F70A0DD7
:104CF0001B1D065A1A4FF8012081213019F482E059
:104D0000808302C0223011F0FF243CC0A0E0B0E05C
:104D10002091CC043091CD044091CE045091CF0429
:104D2000820F931FA41FB51FF80185879687A78759
:104D3000B08B2581368180917E0590917F05281763
:104D40003907B1F480E1B80140E050E00E944C2303
:104D5000F82EC6010E942E24F501EE57F84F8081EF
:104D60009181019779F4C6010E94C145F82E0AC0CD
:104D700081E1B80140E050E00E944C23F82E83E02E
:104D8000F80180838F2DF82E43C094FF40C0C601E8
:104D9000880F991F8C0173E0000F111F7A95E1F7BE
:104DA000080F191F065A1A4FF8018081813011F43B
:104DB00082E022C08230E1F48091CA049091CB0459
:104DC000892B59F080E1B80140E050E00E944C236B
:104DD000F82EC6010E942E241BC081E1B80140E0DC
:104DE00050E00E944C23F82E83E0F801808310C02D
:104DF000833021F486E0F801808309C0853039F4DE
:104E0000C6010E94AB2403C068E0F62E01C0FF2457
:104E10008F2DA696E0E10C943D63CF93DF93089627
:104E20009093B5048093B40482E290E00E949C16B3
:104E30008091C6049091C7040E94D7158091C40444
:104E40009091C5040E94D7158091B4049091B50447
:104E50000E94D71580E090E00E94D715609145052B
:104E60007091460580914705909148050E94DB3E70
:104E70006093D0047093D1048093D2049093D304B0
:104E80006091BC047091BD048091BE049091BF04F8
:104E90000E94DB3E6093D4047093D5048093D604C3
:104EA0009093D7041092D80481E18093D904809123
:104EB000B4049091B5040E94D73E9093DB04809394
:104EC000DA044091B4045091B50481E062E270E0EC
:104ED0000E949321EC01009711F4CFEFDFEF88E2FD
:104EE00090E00E949C16CE010E94D71581E10E949D
:104EF000ED21DF91CF910895A0E1B0E0E2E8F7E283
:104F00000C942B63CE01099668E070E00E94B31503
:104F100089859A850E94D73E9093C5048093C404E6
:104F20008B859C850E94D73E9093C7048093C604CE
:104F30008D859E850E94D73E8C01085010401093AD
:104F4000CB040093CA04085F1F4F80915305E82EDD
:104F5000FF248EE090E0E80EF91E8F859889892B5A
:104F6000B9F16091BC047091BD048091BE04909130
:104F7000BF040E94DB3E6093D0047093D104809301
:104F8000D2049093D3046091C0047091C1048091C5
:104F9000C2049091C3040E94DB3E6093D4047093DA
:104FA000D5048093D6049093D7041092D80481E15D
:104FB0008093D9048D859E859093DB048093DA04D9
:104FC00080E0B701A8010E949321892B09F04AC013
:104FD000C70108969093C9048093C8042091C60421
:104FE0003091C7042B37310519F40E9469343DC054
:104FF0002532310519F40E94263C37C044E02030A8
:10500000340719F40E94DB2D30C02434310519F423
:105010000E949B2B2AC02938310519F40E94232FA6
:1050200024C02151374201F50E9477168E010F5F8F
:105030001F4FC80167E070E00E94B315C80168EE19
:1050400070E047E050E00E949663892B69F48AE2A1
:1050500090E00E949C168FED90E00E94CE180E9476
:105060000D27FFCF89E001C080E06096E6E00C9458
:1050700047638091450890914608A0914708B091F8
:1050800048088093BC049093BD04A093BE04B093E1
:10509000BF0483E490E09093C5048093C40484E447
:1050A00090E09093C7048093C6048AE290E00E9447
:1050B0009C1660E076E081E091E00E94E8150E9495
:1050C000663E6093590870935A0880935B089093EA
:1050D0005C080E94E81580E090E00E94D71580E00F
:1050E00090E00E94D71560E070E080E090E00E94C0
:1050F000E81580E06CE070E00E94191680E091E015
:1051000066E070E00E94011680E06AEC70E00E94A8
:10511000191663E673E582E893E60E94E81581E0DC
:1051200095E30E94D71584E00E94CA1582E30E948D
:10513000CA1584E00E94CA15609145057091460524
:1051400080914705909148050E94E81586E30E94EA
:10515000CA1584E00E94CA156091450870914608FE
:1051600080914708909148080E94E8158FEF0E94AF
:10517000CA1580E06CE270E00E9419168CE291E0A2
:105180000E940D2708950F931F9381E0809370086C
:105190008FEF9FEFAFEFBFEF8093BC049093BD0400
:1051A000A093BE04B093BF0483E490E09093C50441
:1051B0008093C40484E490E09093C7048093C60471
:1051C0001092490510924A0510924B0510924C0519
:1051D0001092450510924605109247051092480519
:1051E0001092F9091092FA091092FB091092FC0929
:1051F00010924D0510924E0510924F0510925005D9
:1052000010924108109242081092430810924408EC
:1052100010923D0810923E0810923F0810924008EC
:105220001092490810924A0810924B0810924C08AC
:1052300010924508109246081092470810924808AC
:10524000109255081092560810925708109258085C
:1052500010924D0810924E0810924F08109250086C
:10526000109251081092520810925308109254084C
:1052700010926508109266081092670810926808EC
:10528000109273080E94663E6093590870935A0802
:1052900080935B0890935C088AE290E00E949C16E1
:1052A00060E076E081E091E00E94E81560915908A5
:1052B00070915A0880915B0890915C080E94E815F3
:1052C00060E070E880E090E00E94E81580E060E136
:1052D00070E00E94191600E011E0C80166E070E07D
:1052E0000E94011680E06AEC70E00E94191663E6E5
:1052F00073E582E893E60E94E81581E095E30E9459
:10530000D71581E00E94CA158DE30E94CA1587E077
:105310000E94CA1581E00E94CA15C80166E070E0CB
:105320000E9401168FEF0E94CA1580E06FE270E0C4
:105330000E9419168CE291E00E940D271F910F9197
:1053400008950F931F93182F80937008883129F0C8
:105350008FEF9FEFAFEFBFEF08C0809145089091AE
:105360004608A0914708B09148088093BC049093E8
:10537000BD04A093BE04B093BF04133051F00E944B
:10538000663E6093590870935A0880935B08909327
:105390005C08E9EEF9E001900020E9F73197E95E59
:1053A000F9400E2F0F5F83E490E09093C504809343
:1053B000C40484E490E09093C7048093C6048AE216
:1053C00090E00E949C1660E076E081E091E00E940F
:1053D000E8156091590870915A0880915B08909186
:1053E0005C080E94E81580E090E00E94D715183113
:1053F00019F080E090E802C080E090E00E94D715AC
:10540000609145057091460580914705909148054A
:105410000E94E81580E06CE070E00E94191680E0C0
:1054200091E066E070E00E94011680E06AEC70E0B6
:105430000E94191663E673E582E893E60E94E81578
:1054400081E095E30E94D71583E00E94CA158CE0A5
:105450000E94CA15802F0E94CA1589EE99E0602F1C
:1054600070E00E940116133019F582E30E94CA15FC
:1054700084E00E94CA158091C8049091C9044096A6
:105480000E9477160E9497150E94E81586E30E94F5
:10549000CA1584E00E94CA156091450870914608BB
:1054A00080914708909148080E94E81519E115C0BD
:1054B000163111F015E211C082E30E94CA1584E092
:1054C0000E94CA156091390870913A0880913B0892
:1054D00090913C080E94E8151FE187E30E94CA15DD
:1054E00086E00E94CA1581E00E94CA1583E00E94EE
:1054F000CA1586E00E94CA1583E30E94CA158AE392
:105500000E94CA158BE30E94CA158DE30E94CA153A
:1055100087E00E94CA1581E00E94CA1580E091E0F0
:1055200066E070E00E9401168FEF0E94CA15101B02
:1055300080E0612F70E00E9419168CE291E00E94D9
:105540000D271F910F910895EF92FF920F931F93D4
:105550008091710890917208892B59F4A8E0B1E00C
:10556000EDE1F1E082E101900D928150E1F760E020
:10557000DCC080917008813031F0863121F08831B3
:1055800011F08931D9F5E0906D08F0906E0800E0D7
:1055900010E088E091E06DE171E00E94743FE61A4E
:1055A000F70A080B190BE0926908F0926A08009359
:1055B0006B0810936C081E141F0410061106F4F0FB
:1055C00080917008813049F0863159F480917308D8
:1055D0008F5F80937308833018F00E94C32803C044
:1055E00086E10E94A129682FA8E0B1E0EDE1F1E099
:1055F00082E101900D928150E1F701C060E0E090FE
:105600006508F09066080091670810916808D80155
:10561000C7010196A11DB11D0297A105B10508F4AE
:1056200084C080915D0890915E08A0915F08B09160
:1056300060082091610830916208409163085091A0
:1056400064080097A105B10591F10197A109B1097D
:1056500080935D0890935E08A0935F08B093600804
:105660002150304040405040209361083093620800
:1056700040936308509364080894E108F108010915
:105680001109E0926508F09266080093670810938C
:1056900068080097A105B10509F047C088E10E949C
:1056A000A129682F882309F040C06CE03EC008940F
:1056B000E108F108010911092115310541055105DC
:1056C00009F1DA01C9010197A109B10980936108C3
:1056D00090936208A0936308B0936408E092650811
:1056E000F092660800936708109368080097A10578
:1056F000B105D9F489E10E94A129682F8823A9F472
:105700006DE013C0E0926508F092660800936708A8
:1057100010936808E114F1040105110531F40E94A9
:10572000C328682F882309F46EE0862F1F910F91FC
:10573000FF90EF900895ACE1B0E0E1EAFBE20C9459
:105740002B6380917008882309F4E8C1873109F43C
:10575000E5C18091C8049091C90480519F4F0E9477
:1057600077160E947815182F8F3F09F4C5C00E9444
:105770007815082F153341F4813009F0D6C10E9405
:10578000781580936F08EDCF113071F4843009F0F3
:10579000CCC10E94971560933D0870933E0880939A
:1057A0003F0890934008DDCF133071F4843008F443
:1057B000BCC10E9497156093410870934208809382
:1057C0004308909344081FC0163371F4843008F4E2
:1057D000ACC10E949715609345087093460880936A
:1057E0004708909348080FC01630A1F4843008F49D
:1057F0009CC10E9497156093490870934A08809352
:105800004B0890934C08043009F4ABCF802F90E004
:1058100004976FC0133309F04BC0843009F0A1CF57
:105820000E9497157B018C01609355087093560870
:10583000809357089093580880915108909152088E
:10584000A0915308B09154080097A105B105B1F497
:10585000C801B7012BE633E040E050E00E94A362AC
:1058600028EE33E040E050E00E94E26220935108CD
:1058700030935208409353085093540880914D0838
:1058800090914E08A0914F08B09150080097A10543
:10589000B10509F066CF16950795F794E794E09265
:1058A0004D08F0924E0800934F081093500859CFBE
:1058B0001A3371F4843009F054CF0E949715609325
:1058C0004D0870934E0880934F089093500849CF2D
:1058D0001B3371F4843009F044CF0E949715609314
:1058E000510870935208809353089093540839CF0D
:1058F00090E00E94BB1835CF8091C8049091C904F4
:1059000004960E9477168091700890916F088130FC
:10591000B9F4923009F004C10E94971520915908FA
:1059200030915A0840915B0850915C0862177307E8
:105930008407950709F0F4C083E00E94A129F1C013
:10594000953009F0D9C00E949715209159083091DF
:105950005A0840915B0850915C08621773078407EE
:10596000950709F0DDC087E1809370088091C80435
:105970009091C90440960E9477160E949715AB013A
:10598000BC014093450550934605609347057093CD
:10599000480588E090E00E94616480913D08909104
:1059A0003E08A0913F08B09140088093490590932C
:1059B0004A05A0934B05B0934C0580914108909106
:1059C0004208A0914308B091440880934D059093FC
:1059D0004E05A0934F05B0935005809149089091D2
:1059E0004A08A0914B08B0914C088093F909909314
:1059F000FA09A093FB09B093FC0980914D0890919E
:105A00004E08A0914F08B091500880935D08909384
:105A10005E08A0935F08B093600880915108909150
:105A20005208A0915308B091540880936108909354
:105A30006208A0936308B093640880915508909120
:105A40005608A0915708B091580880936508909324
:105A50006608A0936708B09368088F5F9F4FAF4FA9
:105A6000BF4F21F41092720810927108DE01119656
:105A7000E4EBF4E08CE101900D928150E1F760914C
:105A800045057091460580914705909148050E9413
:105A90000E1F0E94B6160E94631B8C01A8950E94DF
:105AA000D820813019F40E94B61609C0823039F42A
:105AB0000E9439288823B1F40E94C32813C00E9491
:105AC000631B801B910B8D54914040F38091FD0925
:105AD0008150823030F481E090E09093050A809309
:105AE000040A80E0A4EBB4E0FE0131969CE1019051
:105AF0000D929150E1F715C0963091F40E949715E0
:105B00002091590830915A0840915B0850915C08E7
:105B1000621773078407950719F407C080E001C076
:105B20008FE06C96E6E00C9447630E94C328F9CF9F
:105B3000AF92BF92DF92EF92FF920F931F93DF938A
:105B4000CF930F92CDB7DEB7F82EE92E9C01590105
:105B50008EE2D82E0E947815982F882331F408946D
:105B6000A108B108F501108219C0807C803C11F0B9
:105B700085010AC00E94781511C099830E9478158A
:105B8000F80181938F019981802F8A198917A8F3D1
:105B9000A90EB11CF501D1925F01DCCF8F2D9E2D96
:105BA0000F90CF91DF911F910F91FF90EF90DF90B9
:105BB000BF90AF900895ACE4B0E0E1EEFDE20C944C
:105BC00021638091C8049091C9040E947716CE0188
:105BD00001966CE070E00E94B31589819A810E9461
:105BE000D73E2091DE093091DF098217930709F033
:105BF0006AC08D819E810E94D73E6C01EE24FF24F5
:105C00003DE2A32EB12CAC0EBD1E2DE0822E912CB8
:105C10008C0E9D1E14C0C5010E94982D0E948515F2
:105C20008C010E9485150130110531F4019721F492
:105C3000C401B5010E94FF630894E11CF11CEC143F
:105C4000FD0448F38F8198850E94D73E3C01EE24E5
:105C5000FF249DE2492E512C4C0E5D1E31C0C20125
:105C60000E94982D0E9485158C010E9485154C017B
:105C70000E9497155B016C010E948515013011058A
:105C8000D1F421E082169104B1F48430910599F4A5
:105C90000E949715AB01BC014093E0095093E109C4
:105CA0006093E2097093E309CE010D969601850198
:105CB0000E94013208C00E94BB180894E11CF11C2C
:105CC000E614F70460F280E0C45BDF4FE0E10C947F
:105CD0003D63AF92BF92DF92EF92FF920F931F93BB
:105CE000CF93DF93182F092F8091F9099091FA092A
:105CF000A091FB09B091FC098093BC049093BD0472
:105D0000A093BE04B093BF0485E390E09093C504D4
:105D10008093C40480E094E09093C7048093C60409
:105D20000E94663E7093DF096093DE098AE290E08C
:105D30000E949C168091DE099091DF090E94D71580
:105D400080E091E00E94D71581E090E00E94D71595
:105D500080E090E00E94D71580E090E00E94D71587
:105D600080E090E00E94D715212F302FC901EC016F
:105D700040E1A42EB12C7E010E2D0C1BF701D0802A
:105D8000FEE2DF1631F0DD2021F00894E11CF11C69
:105D9000F3CF802F0E94CA1510E0CE01B8010E94F7
:105DA00001160F5F1F4FA00EB11EDD2019F0E70195
:105DB0002196E1CF80E00E94CA1581E090E00E9428
:105DC000D71581E090E00E94D715C50101960E9489
:105DD0000D27DF91CF911F910F91FF90EF90DF90F2
:105DE000BF90AF9008951F930E947815182F1154FB
:105DF0001295107F0E94781581548F70812B1F910E
:105E000008950F931F93CF93DF93EC0100E08991E6
:105E100090E00E946A63182F8595859585958595F4
:105E20008F5B0E94CA151F70812F8F5B0E94CA155D
:105E30000F5F003161F780E00E94CA15DF91CF91BA
:105E40001F910F910895ACE1B0E0E9E2FFE20C94FC
:105E500021638091C8049091C9040E947716CE01F5
:105E600001966CE070E00E94B3158B819C810E94CA
:105E7000D73E9C018F709070892B11F082E1EEC0AB
:105E800037FF5AC089819A810E94D73E2091DE094E
:105E90003091DF098217930709F0DFC08F81988561
:105EA0000E94D73E019711F080E1D8C00E9478157A
:105EB000803211F081E1D2C08E01035F1F4FC80113
:105EC000902E892E2DE1E22EF12CEC0EFD1E0E946B
:105ED000F32EF80181938F01EE15FF05C1F71C8E9B
:105EE0000E9478150E9485158C010E9485157C0101
:105EF0000E9497155B016C010032110509F0ADC0DD
:105F0000F1E0EF16F10409F0A8C00E9485150E9487
:105F100085150E949715AB01BC014093E009509391
:105F2000E1096093E2097093E309892D982D9601A8
:105F300085010E94013291C020703877232B09F02F
:105F40008CC08091CA049091CB04C29709F085C09F
:105F500089819A810E94D73E4C018D819E810E9449
:105F6000D73E5C01CC24DD249DE0692E712C6C0EA3
:105F70007D1E8DE1482E512C4C0E5D1E31C00E94BD
:105F80007815803209F069C083010E94F32EF80170
:105F900081938F01E415F505C1F71C8E0E947815D9
:105FA0000E9485157C010E9485150197B1F4F0E2ED
:105FB000EF16F10451F4C30169EE79E00E94F66333
:105FC000009759F400E015E84FC081E2E816F104AB
:105FD00021F48D858A3209F445C00894C11CD11C76
:105FE000CA14DB0460F239C086E090E00E94D71545
:105FF00080E090E00E94D7156091450570914605BC
:1060000080914705909148050E94E8158EE390E045
:1060100021C08DE390E00E94D71581E00E94CA154F
:1060200089EE99E06FE070E00E94011680E00E9426
:10603000CA1580E094E00E94D71580E091E066E008
:1060400070E00E94011680E064E270E00E94191680
:1060500085E790E00E940D2701C080E06C96E0E1AA
:106060000C943D6300E014E88AE290E00E949C16E4
:10607000C4010E94D715C8010E94D71580E090E0A6
:106080000E94D71581E090E00E94D71580E090E053
:106090000E94D71580E090E00E94D71580E20E9410
:1060A000CA15CE010D960E94012FC7010E94D71577
:1060B00081E090E00E94D71568E572E080E090E012
:1060C0000E94E815E0E2EE16F10409F0A2CF8CCFB1
:1060D0000F931F938C018091490590914A05A091DF
:1060E0004B05B0914C0580959095A095B095209169
:1060F0004505309146054091470550914805822B52
:10610000932BA42BB52B8093BC049093BD04A09338
:10611000BE04B093BF0489E890E09093C5048093D7
:10612000C4049093C7048093C6040E94663E709393
:10613000DF096093DE098AE290E00E949C1680915C
:10614000DE099091DF090E94D71580E191E00E945D
:10615000D71581E090E00E94D71580E090E00E9482
:10616000D71580E090E00E94D71580E090E00E9473
:10617000D71580E20E94CA15C8010E94012F80E253
:1061800090E00E94D71581E090E00E94D71582E34D
:1061900090E00E940D271F910F910895E8EBF8E021
:1061A00084818130A1F480819181A281B3810097A3
:1061B000A105B10561F00197A109B109808391831F
:1061C000A283B3830097A105B10509F41482B9969F
:1061D0008AE0E030F80721F70895A9E2B0E0E3EFA4
:1061E000F0E30C9429637C0104E918E06E01089443
:1061F000C11CD11CD601F80189E201900D92815099
:10620000E1F789A5813059F4C601B7010E94F66310
:10621000009729F429A13AA14BA15CA10AC0075D0E
:106220001F4F89E00C3D180729F720E030E040E0DF
:1062300050E0B901CA01A996E8E00C944563CF93F8
:10624000DF938091E609813001F5C4E7D8E0CE0103
:1062500060EE79E00E94E13E813009F4C3C0FE01A6
:1062600001900020E9F73197EC1BFD0B709738F493
:10627000CE016EE270E00E94EB63009711F084E0C3
:1062800001C082E08093E609A9C0823009F584E765
:1062900098E00E94ED306093E0097093E1098093EB
:1062A000E2099093E309611571058105910509F0F3
:1062B00099C00E94631B9093DD098093DC0984E7F9
:1062C00098E00E946830282F1092E50983E053C0BF
:1062D000833079F58091E0099091E109A091E2097C
:1062E000B091E3090097A105B10509F07BC00E94B8
:1062F000631B2091DC093091DD09821B930B885EC2
:10630000934008F46BC08091E5098F5F8093E509A5
:10631000833020F020910C082D5E61C00E94631B29
:106320009093DD098093DC0984E798E00E9468304F
:1063300053C0843019F584E798E00E94ED306093F3
:10634000E0097093E1098093E2099093E3096115F4
:1063500071058105910509F045C00E94631B90936A
:10636000DD098093DC0984E798E00E94692E282FDC
:106370001092E50985E08093E60931C0853071F51A
:106380008091E0099091E109A091E209B091E309BF
:106390000097A105B10531F50E94631B2091DC092E
:1063A0003091DD09821B930B885E9340B8F0809199
:1063B000E5098F5F8093E509833020F020910C0878
:1063C000295E0DC00E94631B9093DD098093DC0958
:1063D00084E798E00E94692E282F01C020E080E029
:1063E00090E003C020E081E090E09093E809809382
:1063F000E709019711F41092E609822FDF91CF91FE
:106400000895A0E0B0E0E7E0F2E30C942363EC0130
:106410006A017B014801590100E010E089E2682E21
:10642000712C069DC001079D900D169D900D1124A5
:106430008C56974FBE010E94F663009739F10F5FAB
:106440001F4F0830110569F72091E409822F8F5FF3
:1064500087708093E40930E089E290E0289F800112
:10646000299F100D389F100D11240C56174FC8018D
:10647000BE010E94FF63F801C0A2D1A2E2A2F3A272
:1064800084A295A2A6A2B7A281E080A7CDB7DEB76D
:10649000EEE00C943F63A8E0B0E0E1E5F2E30C9499
:1064A00027636D837E838F83988719821A821B826C
:1064B0001C8229813A814B815C81F8EEAF2EE3E0AA
:1064C000BE2ECC24DD24EE24FF2400E010E00E9448
:1064D0002E5C952FB901842F2896EAE00C94436333
:1064E000A4E2B0E0E6E7F2E30C94296310910C0813
:1064F00010930D0800E0B5E0EB2EF12CEC0EFD1E24
:106500006E010894C11CD11C1F5F1370E12FF0E0D5
:10651000EE0FFF1FEC5AFE4F65917491C7010E9468
:10652000FF63C701B6010E94E13E813041F48981D9
:106530009A81AB81BC810097A105B10519F0109338
:106540000C0803C00F5F0430F9F6A496E8E00C9441
:106550004563AF92BF92CF92DF92EF92FF920F937B
:106560001F936093BC047093BD048093BE0490930A
:10657000BF048BE790E09093C5048093C40490938C
:10658000C7048093C6048AE290E00E949C1683E2CE
:106590000E94CA1580E067E270E00E941916F89424
:1065A000E0908D01F0908E0100918F01109190018B
:1065B0006091190C70911A0C882777FD8095982F9F
:1065C0000E944B325B016C01789460931E087093BB
:1065D0001F08809320089093210880E89EE7AAEA8C
:1065E000B3E8E80EF91E0A1F1B1FC801B7010E947D
:1065F000E815C601B5010E94E81580E390E00E940D
:106600000D271F910F91FF90EF90DF90CF90BF90DB
:10661000AF9008951F9310910E0A112309F480C0C2
:106620001130A1F480910C08E82FF0E0EE0FFF1F6D
:10663000EC5AFE4F6591749184E798E00E94FF63E5
:106640001093E60982E080930E0A6AC0123089F541
:106650008091E7099091E809019709F061C01092D3
:10666000E8091092E7096091E0097091E1098091D1
:10667000E2099091E30960938807709389078093FA
:106680008A0790938B07109236080E94A932182F20
:10669000882351F483E080930E0A0E94631B909339
:1066A0002F0880932E0802C010920E0A0E947032AA
:1066B00038C01330A9F50E94631B20912E08309139
:1066C0002F08821B930B20913008309131088217DC
:1066D000930730F1809136088F5F809336088330BE
:1066E00040F01093930110910D08145E0E94B60BB8
:1066F00018C0609188077091890780918A079091EE
:106700008B070E94A932182F882339F40E94631B3B
:1067100090932F0880932E0804C010920E0A01C097
:1067200010E0812F1F9108958091FF0987708230BA
:1067300019F484EF90E004C0833041F480EF90E0DE
:106740000E94CE1880E00E94CA1508956091450508
:106750007091460580914705909148050E94E81583
:106760000895AF92BF92CF92DF92EF92FF920F9374
:106770001F938091120890911308A0911408B09172
:1067800015088093BC049093BD04A093BE04B093FD
:10679000BF048BE790E09093C5048093C40490936A
:1067A000C7048093C60480910F0A9091100A892B28
:1067B00019F405EE10E102C005E211E08AE290E072
:1067C0000E949C16802F0E94CA15812F0E94CA1514
:1067D000609132087091330820E030E84FE0C90141
:1067E00086239723892B29F4415019F03695279554
:1067F000F6CF842F0E94CA1586EF0E94CA156091B9
:1068000016087091170880911808909119080E9435
:10681000E81560911A0870911B0880911C089091EE
:106820001D080E94E8150E94943360912C08709115
:106830002D0880E090E00E944B327B018C0160913A
:10684000260870912708809128089091290860589F
:10685000714885459C470E94E815C801B7010E9410
:10686000E81580E060E170E00E941916F894E0906D
:106870008D01F0908E0100918F0110919001609137
:10688000190C70911A0C882777FD8095982F0E941B
:106890004B325B016C01789480E89EE7AAEAB3E88A
:1068A000E80EF91E0A1F1B1FC801B7010E94E81558
:1068B000C601B5010E94E81580E390E00E940D2713
:1068C0001F910F91FF90EF90DF90CF90BF90AF900E
:1068D0000895A7E6B0E0EFE6F4E30C941F6380911F
:1068E000C8049091C9040E947716CE01819660E396
:1068F00070E00E94B31599A1892F8770843009F048
:106900001CC480910E0A882309F49AC7892F807CC1
:10691000809306019AA1803C21F0992311F09031D7
:1069200058F082E0809393011092E60910920E0ACB
:106930000E94B60B8BE185C79F5F909307016DA105
:106940007EA18FA198A50E94DB3E609316087093EC
:106950001708809318089093190869A57AA58BA544
:106960009CA50E94DB3E60931A0870931B088093DD
:106970001C0890931D08FE01E05CFF4F90812FAD35
:106980005EAD6DAD7CADABADDAAC99ACFE01EC5B50
:10699000FF4FC080FE01ED5BFF4FB080FE01EE5B5C
:1069A000FF4FA080FE01EF5BFF4F7080FE01E85BB0
:1069B000FF4F8081FE01E95BFF4F3081FE01EA5B02
:1069C000FF4F4081FE01EB5BFF4FE081E82EE91AAB
:1069D00091E08E1508F090E0832F821B21E038179C
:1069E00008F020E0F82EF91A91E08F1508F090E0F9
:1069F000292B842F851B31E0481708F030E0082F41
:106A0000021B91E0801708F090E0392B8E2F861B37
:106A100021E0E81708F020E0182F131B91E0811700
:106A200008F090E0292B8C2D871B31E0C81608F068
:106A300030E0B82FB21B91E08B1708F090E0392BB3
:106A40008B2D8A1B21E0B81608F020E0A82FA31B8D
:106A500091E08A1708F090E0292B8A2D8D1991E09A
:106A6000A81608F090E0F82FF21B21E08F1708F02D
:106A700020E0922BE72DE919E91B9701A8016B2F64
:106A80007A2F8F2F9E2F52F52E2D2F5F81E02E15FE
:106A900008F080E0382F3F0D81E03F1508F080E0DE
:106AA000482F400F81E0401708F080E0582F510F29
:106AB00081E0511708F080E0682F6B0F81E06B17C1
:106AC00008F080E0782F7A0F81E07A1708F080E0F4
:106AD0008F0F91E08F1708F090E09E0F01E00E9469
:106AE000A95B622E532E442E352E262E62967FAF42
:106AF000629763968FAF639764969FAF6497FE012A
:106B0000E45BFF4FC080FE01E55BFF4FB080FE01FC
:106B1000E65BFF4FA080FE01E75BFF4F7080FE0148
:106B2000E05BFF4F0081FE01E15BFF4FF080FE0163
:106B3000E25BFF4F9080FE01E35BFF4F808080911E
:106B4000220890912308A0912408B091250880582C
:106B50009148A545BC47182F8D8B9E8BAF8BB88F66
:106B600060912A0870912B0880E090E00E944B32DF
:106B7000698B7A8B8B8B9C8B872F3B89492F5E8906
:106B80007F89E88DD02ED61A91E00D1508F090E09F
:106B90002F2D281B822F21E0F81608F020E0E82E88
:106BA000E91A91E08E1508F090E0292B892D831BBE
:106BB00031E0981608F030E0F82EF21A91E08F15C7
:106BC00008F090E0392B882D841B21E0881608F00E
:106BD00020E0082F031B91E0801708F090E0292B9C
:106BE0003C2D311B132F91E0C31608F090E0B12F1C
:106BF000B21B81E01B1708F080E0982B8B2D851BC2
:106C000021E0B81608F020E0A82FA91B91E08A1710
:106C100008F090E0292B8A2D871B91E0A81608F038
:106C200090E0F82FF21B21E08F1708F020E0922B64
:106C30007E1AE72DE91B2D2D3E2D4F2D502F6B2F4A
:106C40007A2F8F2F9E2F52F52D2D2F5F81E02D153E
:106C500008F080E0382F3E0D81E03E1508F080E01E
:106C6000482F4F0D81E04F1508F080E0582F500F4E
:106C700081E0501708F080E0682F6B0F81E06B1700
:106C800008F080E0782F7A0F81E07A1708F080E032
:106C90008F0F91E08F1708F090E09E0F01E00E94A7
:106CA000A95BA32FB42F152F062FF72ED82EC22E97
:106CB000C60CF1E0C21608F0F0E03A2F350DE1E025
:106CC0003A1708F0E0E0EF2EE30E21E0E31608F0BB
:106CD00020E0E22B4B2F440D31E04B1708F030E061
:106CE000AE2FA40F21E0A41708F020E0322B512F83
:106CF000530D41E0511708F040E0F32FF50F21E06C
:106D0000F51708F020E0422B602F620D31E060178C
:106D100008F030E0E42FE60F21E0E61708F020E06D
:106D2000322B62967FAD62977F0D41E07F1508F0B0
:106D300040E0532F570F21E0571708F020E0422B77
:106D400063968FAD63978D0D21E08D1508F020E0DF
:106D5000480F31E0481708F030E0232B64968FADE0
:106D60006497980F290FC98AEA8AAB8BFC8BED8B4D
:106D70005E8B4F8B288F4D885E886F88788C8989D1
:106D80009A89AB89BC894C015D01CC24DD24760154
:106D90009C01A50160E070E080E090E002E00E94CC
:106DA0002A5B122F232E65964FAF659766965FAFCD
:106DB000669767966FAF679768967FAF6897699693
:106DC0008FAF69976A969FAF6A9705E00E942A5B2A
:106DD000A32FB42F052F6B966FAF6B976C967FAF79
:106DE0006C976D968FAF6D976E969FAF6E97322EA4
:106DF000311AF1E0231508F0F0E03A2F3219E1E002
:106E0000A31708F0E0E0132F1F1B21E0311708F053
:106E100020E0E22B4B2F65969FAD6597491B31E033
:106E2000B41708F030E0B42FBE1B21E04B1708F078
:106E300020E0322B502F6696AFAD66975A1B41E08B
:106E4000051708F040E0052F031B21E0501708F05C
:106E500020E0422B6B966FAD6B976796EFAD67970F
:106E60006E1B31E06B96FFAD6B97F61708F030E0C4
:106E7000962F941B21E0691708F020E0322B6C96C6
:106E80007FAD6C9768962FAD6897721B41E06C964A
:106E90008FAD6C97871708F040E0A72FA31B21E068
:106EA0007A1708F020E0422B6D968FAD6D976996AA
:106EB000EFAD69978E1B21E06D96FFAD6D97F817CA
:106EC00008F020E0E82FE41B31E08E1708F030E0F6
:106ED000232B6E96FFAD6E976A963FAD6A97F31BB4
:106EE000F21B232C280C31E0231408F030E0812F12
:106EF000890D41E0811708F040E0380F51E0381764
:106F000008F050E0452B8B2F8A0D51E08B1708F0CD
:106F100050E0480F61E0481708F060E0562B202F42
:106F20002B0D81E0201708F080E0520F61E052172E
:106F300008F060E0682B690F71E0691708F070E0F5
:106F40007A0F81E07A1708F080E08E0F91E08E17BB
:106F500008F090E0222D9F0F03E00E942A5B298F0A
:106F60003A8F4B8F5C8F6D8F7E8F8F8F98A3ED8CB8
:106F7000FE8C0F8D18A180911B0190911C01892B13
:106F8000C9F48091370890913808009799F0A301CF
:106F9000920177FE07C022273327A901241935095A
:106FA00046095709A0E0B0E082179307A407B50788
:106FB0000CF446C48701F89480918D0190918E0164
:106FC000A0918F01B0919001840D951DA61DB71D54
:106FD00080938D0190938E01A0938F01B0939001C7
:106FE0008091190C90911A0C8E0D9F1D90931A0C84
:106FF0008093190C8091190C90911A0C97FF2AC05C
:1070000080918D0190918E01A0918F01B09190019E
:10701000181619061A061B06ECF480918D01909142
:107020008E01A0918F01B09190010197A109B10942
:1070300080938D0190938E01A0938F01B093900166
:107040008091190C90911A0C88519C4F90931A0CB6
:107050008093190C80918D0190918E01A0918F01E8
:10706000B09190018093260890932708A093280858
:10707000B09329088091190C90911A0C90932D08C7
:1070800080932C08789477FE0AC0101611063CF401
:107090000894411C511C611C711C085E1340D301F3
:1070A000C20180509048AF4FBF4F80509040A140E8
:1070B000B04038F08FEF9FE790930F0880930E0851
:1070C00004C050920F0840920E08109311080093CC
:1070D00010088091170A882361F1C301B20128EEDC
:1070E00033E040E050E00E94A3629B01AC01C80184
:1070F000AA2797FDA095BA2F820F931FA41FB51F33
:10710000B7FD04C0B801620F731F0AC0C301B2010A
:1071100028E13CEF4FEF5FEF0E94A362601B710B11
:107120007093160A6093150A6D54714014F081E053
:1071300001C082E08093170A7DC3833009F0D6C076
:10714000292F287380910F0A9091100A019701F559
:1071500050900601522A40900701E0902608F090D6
:107160002708009128081091290880E89EE7AAEADC
:10717000B3E8E80EF91E0A1F1B1F60912C087091DE
:107180002D0880E090E00E944B323B014C010BC087
:1071900040EC542E522A662477244301EE24FF2427
:1071A000870130E1432EA0902208B0902308C090C0
:1071B0002408D090250820902A0830902B088AE2D5
:1071C00090E00E949C16852D84600E94CA15842D33
:1071D0000E94CA158BA10E94CA1586EF0E94CA158B
:1071E00060E070E080E090E00E94E81560E070E010
:1071F00080E090E00E94E8150E949433C801B70136
:107200000E94E815C401B3010E94E81580910F0A9D
:107210009091100A019799F4CE0181968C01085D36
:107220001F4F20E3E22EF12CE80EF91ED8018D91BC
:107230008D010E94CA150E151F05C1F70CC060E034
:1072400070E080E090E00E94E81560E070E080E08F
:1072500090E00E94E81580E89EE7AAEAB3E8A80E4D
:10726000B91ECA1EDB1EC601B5010E94E815B10198
:1072700080E090E00E944B320E94E81580910F0A56
:107280009091100A019739F0AA24BB246501EE24DD
:10729000FF2487011EC0F894E0908D01F0908E01CC
:1072A00000918F011091900180E89EE7AAEAB3E86F
:1072B000E80EF91E0A1F1B1F6091190C70911A0C21
:1072C000882777FD8095982F0E944B325B016C01D7
:1072D0007894C801B7010E94E815C601B5010E9463
:1072E000E81580E390E00E940D27ABC2853009F0DD
:1072F000A7C28091FF098770813009F0A1C2892F50
:10730000807C809306019AA1803C09F499C299235C
:1073100009F496C2903109F493C29F5F90930701DC
:107320006DA17EA18FA198A50E94DB3E60931608F7
:1073300070931708809318089093190869A57AA587
:107340008BA59CA50E94DB3E60931A0870931B08D6
:1073500080931C0890931D08FE01E05BFF4FD080D6
:10736000FE01E15BFF4FC080FE01E25BFF4FA080AA
:10737000FE01E35BFF4F10813D2DD9822C2DCA8287
:107380009A2DAB82812F1C83FE01E45BFF4FD080DE
:10739000FE01E55BFF4FC080FE01E65BFF4FA08072
:1073A000FE01E75BFF4F1081DD82CE82AF8218873E
:1073B000032FF22EE92EB82E832F822B892B8B29B7
:1073C0008D298C298A29812B09F43AC2F89480915D
:1073D0008D0190918E01A0918F01B0919001805804
:1073E0009148A545BC478D839E83AF83B887609144
:1073F000190C70911A0C882777FD8095982F0E94A0
:107400004B3269837A838B839C83789489812A8128
:107410003B814C815D81AE81BF819884F02FF81B48
:1074200091E00F1708F090E08F2D821B21E0F816F5
:1074300008F020E0E82FE91B91E08E1708F090E0BB
:10744000292B8E2D831B31E0E81608F030E0782FD1
:10745000721B91E0871708F090E0392B8B2D841B6D
:1074600021E0B81608F020E0682F631B91E0861732
:1074700008F090E0292B8D2D851B31E0D81608F0FF
:1074800030E0582F521B91E0851708F090E0392B1F
:107490008C2D8A1B21E0C81608F020E0482F431BE2
:1074A00091E0841708F090E0292B8A2D8B1B91E046
:1074B000A81608F090E0382F321B21E0831708F05F
:1074C00020E0922B1919191BF983EA837B836C83C3
:1074D0005D834E833F8318874D805E806F80788404
:1074E00089819A81AB81BC814C015D01CC24DD2472
:1074F00076019C01A50160E070E080E090E002E090
:107500000E942A5B122F232E6F964FAF6F97A09683
:107510005FAFA097A1966FAFA197A2967FAFA297FA
:10752000A3968FAFA397A4969FAFA49705E00E9460
:107530002A5BA32FB42F052FA5966FAFA597A6960C
:107540007FAFA697A7968FAFA797A8969FAFA8974C
:10755000322E311AF1E0231508F0F0E03A2F3219FB
:10756000E1E0A31708F0E0E0132F1F1B21E0311723
:1075700008F020E0E22B4B2F6F969FAD6F97491BD1
:1075800031E0B41708F030E0B42FBE1B21E04B17F8
:1075900008F020E0322B502FA096AFADA0975A1BD9
:1075A00041E0051708F040E0052F031B21E05017CC
:1075B00008F020E0422BA5966FADA597A196EFAD00
:1075C000A1976E1B31E0A596FFADA597F61708F0C1
:1075D00030E0962F941B21E0691708F020E0322B51
:1075E000A6967FADA697A2962FADA297721B41E0FB
:1075F000A6968FADA697871708F040E0A72FA31B8C
:1076000021E07A1708F020E0422BA7968FADA797CC
:10761000A396EFADA3978E1B21E0A796FFADA7978A
:10762000F81708F020E0E82FE41B31E08E1708F08F
:1076300030E0232BA896FFADA897A4963FADA49762
:10764000F31BF21B232C280C31E0231408F030E04C
:10765000812F890D41E0811708F040E0380F51E09B
:10766000381708F050E0452B8B2F8A0D51E08B170F
:1076700008F050E0480F61E0481708F060E0562B32
:10768000202F2B0D81E0201708F080E0520F61E0E1
:10769000521708F060E0682B690F71E0691708F075
:1076A00070E07A0F81E07A1708F080E08E0F91E0A9
:1076B0008E1708F090E0222D9F0F03E00E942A5BB6
:1076C00029873A874B875C876D877E878F87988B62
:1076D000ED84FE840F85188980911B0190911C0117
:1076E000892BC9F48091370890913808009799F058
:1076F000A301920177FE07C022273327A90124198D
:10770000350946095709A0E0B0E082179307A4079E
:10771000B5070CF495C09701F89480918D01909174
:107720008E01A0918F01B0919001840D951DA61D31
:10773000B71D80938D0190938E01A0938F01B0931C
:1077400090018091190C90911A0C8E0D9F1D9093B1
:107750001A0C8093190C8091190C90911A0C97FFB8
:107760002AC080918D0190918E01A0918F01B091DE
:107770009001181619061A061B06ECF480918D016B
:1077800090918E01A0918F01B09190010197A10974
:10779000B10980938D0190938E01A0938F01B093D6
:1077A00090018091190C90911A0C88519C4F9093E4
:1077B0001A0C8093190C80918D0190918E01A091EB
:1077C0008F01B09190018093260890932708A09391
:1077D0002808B09329088091190C90911A0C909365
:1077E0002D0880932C08789477FE0AC01216130691
:1077F0003CF40894411C511C611C711C285E3340F0
:10780000D301C20180509048AF4FBF4F805090408D
:10781000A140B04038F08FEF9FE790930F0880931E
:107820000E0804C050920F0840920E0830931108C1
:107830002093100881E090E090931E0C80931D0C23
:1078400080E0C959DF4FE2E10C943B6380910F0A5D
:107850009091100A892B11F480E008958AE290E05B
:107860000E949C16F89460918D0170918E01809118
:107870008F019091900178946058714885459C479C
:107880000E94E81584E090E00E940D270895DB0136
:10789000982F92959F702CE531E0F901E90FF11DC9
:1078A000E491EC938F70280F311DF90184911196AA
:1078B0008C93119712961C921297CB010895DB01BD
:1078C000292F22952F704CE551E0FA01E20FF11DAE
:1078D000E491EC939F70FA01E90FF11DE491119688
:1078E000EC931197982F92959F70FA01E90FF11D73
:1078F000E4911296EC9312978F70480F511DFA0184
:10790000849113968C93139714961C921497CB0121
:107910000895DA01292F22952F704CE551E0FA01E4
:10792000E20FF11DE491EC939F70FA01E90FF11D54
:10793000E4911196EC931197982F92959F70FA010C
:10794000E90FF11DE4911296EC9312978F70FA01F2
:10795000E80FF11DE4911396EC931397872F82950E
:107960008F70FA01E80FF11DE4911496EC931497CF
:107970007F70FA01E70FF11DE4911596EC931597CE
:10798000862F82958F70FA01E80FF11DE49116960B
:10799000EC9316976F70460F511DFA01849117965C
:1079A0008C93179718961C921897CD010895282F3D
:1079B000DB0164E60E94C262392F822F0E94C262FC
:1079C000805DFD018193832F6AE00E94C262805D29
:1079D00011968C931197832F0E94C262905D9183C0
:1079E0001282CD010895A0E0B0E0E9EFFCE30C9431
:1079F0002A63482FF92EE62ED72E862F972F9C012B
:107A0000E901E0E1F7E200E010E0842F9F2DBF01E3
:107A10000E94CE62262F842F9F2DBF010E94CE622E
:107A2000482FF92E205D2993CF016AE070E00E9473
:107A3000CE62FB010F5F1F4F0430110531F7405D2F
:107A4000488319828E2D9D2DCDB7DEB7E7E00C94CB
:107A50004663A0E0B0E0EFE2FDE30C942263062F62
:107A6000772E4C01642E552E842F952F9C01E90111
:107A7000C12C8AECD82E8AE9E82E8BE3F82EAA24B2
:107A8000BB24602F772DC401A70196010E94E262FA
:107A9000122F602F772DC401A70196010E94E26288
:107AA000062F772E4C01105D1993C701B6012AE00D
:107AB00030E040E050E00E94E262C901DA016C016E
:107AC0007D010894A11CB11C89E0A816B104C9F677
:107AD000005D08831982862D952DCDB7DEB7EFE0C6
:107AE0000C943E63EF92FF920F931F938B019C01C6
:107AF000F42EE52E97FD04C0842F952FFC010CC0B9
:107B000030952095109501951F4F2F4F3F4F842F93
:107B1000952FFC018DE28193C901B801AF010E944C
:107B2000293D8F2D9E2D1F910F91FF90EF9008956D
:107B30001F93CF93DF93EC0120E030E040E050E072
:107B40001881812F80538A30C8F4CA01B9012AE014
:107B500030E040E050E00E94A3629B01AC01812F25
:107B6000992787FD9095C097AA2797FDA095BA2FD2
:107B7000280F391F4A1F5B1F2196E2CF203080E07B
:107B8000380781E0480780E0580720F02FEF3FEFEB
:107B900040E050E0C901DF91CF911F910895982FE7
:107BA0008154863010F487E307C0892F81568630D0
:107BB00010F487E501C080E3981B892F0895FF9298
:107BC0000F931F938C01FC0180810E94CF3DF82E02
:107BD000F29490EFF922F80181810E94CF3D8F70DD
:107BE0008F291F910F91FF900895EF92FF920F93AD
:107BF0001F938C01FC0180810E94CF3DF82EF294EE
:107C000030EFF322F80181810E94CF3D8F70F82A76
:107C1000F80182810E94CF3DE82EE29420EFE2221B
:107C2000F80183810E94CF3D8F708E299F2D1F9177
:107C30000F91FF90EF900895CF92DF92EF92FF9215
:107C40000F931F938C01FC0180810E94CF3DC82EB1
:107C5000C29470EFC722F80181810E94CF3D8F70DE
:107C6000C82AF80182810E94CF3DD82ED29460EFBD
:107C7000D622F80183810E94CF3D8F70D82AF80167
:107C800084810E94CF3DF82EF29450EFF522F80146
:107C900085810E94CF3D8F70F82AF80186810E946D
:107CA000CF3DE82EE29440EFE422F80187810E9464
:107CB000CF3D8F708E29682F7F2D8D2D9C2D1F918C
:107CC0000F91FF90EF90DF90CF900895EF92FF9289
:107CD0000F931F938091940190919501A09196012B
:107CE000B09197017C018D012BE0EE0CFF1C001F71
:107CF000111F2A95D1F7E826F9260A271B2780911C
:107D0000980190919901A0919A01B0919B01809363
:107D1000940190939501A0939601B093970180915F
:107D20009C0190919D01A0919E01B0919F01809333
:107D3000980190939901A0939A01B0939B0180912F
:107D4000A0019091A101A091A201B091A301809303
:107D50009C0190939D01A0939E01B0939F019C0173
:107D6000AD01F3E15695479537952795FA95D1F7EB
:107D7000282739274A275B272E253F2540275127CB
:107D8000EF2CF02E012F11272E253F2540275127BC
:107D90002093A0013093A1014093A2015093A3012D
:107DA000B901CA011F910F91FF90EF900895282FFC
:107DB000892F922F0895362F272F692F782FC901E9
:107DC0000895A0E2B0E0E7EEFEE30C9425639C0189
:107DD0005B018E010F5F1F4FC801B9010E94FF6355
:107DE000CC24DD247601980140E1842E912C8C0E68
:107DF0009D1EF80180818E3291F41082C9010E948B
:107E0000983DA0E0B0E08C299D29AE29BF29CC2463
:107E1000D82EE92EFA2E98012F5F3F4F2BC08823D2
:107E2000E9F4CE0101960817190731F4F501108223
:107E300011821282138210C0F8011082C9010E94BF
:107E4000983DA0E0B0E08C299D29AE29BF29F5011D
:107E500080839183A283B38381E013C0992787FD38
:107E60009095C0970A9730F0F50110821182128226
:107E7000138206C00815190519F00F5F1F4FB9CFFF
:107E800080E0A096ECE00C944163CF92DF92EF92F9
:107E9000FF920F931F936B01E82E8A01892FBA017D
:107EA0000E94D73C5EE2F52EF801F382B8016C5FC8
:107EB0007F4F8E2D0E94D73CF801F782B801685F92
:107EC0007F4F8D2D0E94D73CF801F386B801645F87
:107ED0007F4F8C2D0E94D73CC8011F910F91FF90BE
:107EE000EF90DF90CF900895CF92DF92EF92FF92C4
:107EF0000F931F936B010E944A1E7B018C01C601E8
:107F00000E944A1E9B01AC012E193F09400B510BE8
:107F1000B901CA011F910F91FF90EF90DF90CF90B0
:107F20000895A4E0B0E0E7E9FFE30C942D63162F79
:107F3000072F0E944A1E2091890130918A014091A9
:107F40008B0150918C01260F371F481F591F298321
:107F50003A834B835C83CE0101960E94A21EAC0142
:107F6000009711F480E00BC0812F902F9C01D90164
:107F7000FA0182E101900D928150E1F781E02496AF
:107F8000E4E00C944963A4E0B0E0E9ECFFE30C9476
:107F90002963D62EC72E79018A010E944A1E6E19C6
:107FA0007F09800B910B69837A838B839C83CE013D
:107FB00001960E94A21EAC01009711F480E00BC054
:107FC0008D2D9C2D9C01D901FA0182E101900D9229
:107FD0008150E1F781E02496E8E00C944563EF924C
:107FE000FF920F931F93E82EF62E8A01FA940E94B7
:107FF0002D1CF8018083813131F48E2D8F5FF816AE
:1080000060F480E00AC0823111F08E2D06C0EE20AF
:1080100011F48F2D02C08E2D81501F910F91FF9072
:10802000EF900895A0E0B0E0E8E1F0E40C94206364
:10803000C82E362E7A01B22EE8010E94CB1AEB2D03
:10804000FF27E7FDF095EE0DFF1D1082F7019081EF
:10805000892F80538A3010F4182F08C0892F81543B
:10806000863010F010E002C0192F1753A8951B9B03
:10807000FDCF81E00E947E1A219711F08AE001C0B5
:1080800080E1012F112707FD1095DC2CC0E0D0E026
:108090004B2C552447FC5094882E992487FC9094AF
:1080A00034010894610871085701AC0EBD1E8D2D76
:1080B000632D0E94921A0A30110518F4802F805DFA
:1080C00002C0802F895C0E94621A0E94761A0E9468
:1080D0002D1C813141F40F5F1F4F081519054CF01D
:1080E00000E010E006C0823179F40150104017FD25
:1080F00083010A30110518F4802F805D02C0802FA3
:10810000895CF5018083D0CF833151F52196D394DA
:10811000F701EC0FFD1F8081992787FD90950E9444
:108120005663892B11F42196D394C415D5051CF000
:10813000DC2CC0E0D0E0F701EC0FFD1FE0818E2FBA
:1081400080538A3040F08E2F8154863010F080E0CA
:1081500002C08E2F8753082F112707FD1095A4CF3B
:10816000843119F401E010E005C0893109F09CCF99
:1081700000E010E080E00E947E1AC801CDB7DEB7B3
:10818000E1E10C943C638091290C8130C1F5809130
:10819000230C9091240CA091250CB091260C0196F3
:1081A000A11DB11D8093230C9093240CA093250C4A
:1081B000B093260C8091230C9091240CA091250C57
:1081C000B091260C8093260890932708A093280846
:1081D000B093290880938D0190938E01A0938F0115
:1081E000B093900110922D0810922C0881E090E03D
:1081F00090931E0C80931D0C1092290C3EC0809110
:10820000270C823099F080918D0190918E01A09180
:108210008F01B09190010196A11DB11D80938D0138
:1082200090938E01A0938F01B09390018091FF09EC
:108230008770823031F52091000A3091010A2115B2
:108240003105D9F08091210C9091220C01969093E8
:10825000220C8093210C8091210C9091220C82178A
:10826000930778F089E080939301809192018430A4
:1082700041F083E08093920104C01092220C10928E
:10828000210C809192018130C1F48091020A909179
:10829000030A892B91F080911F0C9091200C01977B
:1082A0009093200C80931F0C80911F0C9091200CB8
:1082B000892B19F482E08093920181E090E0909301
:1082C0001C0C80931B0C08951F920F920FB60F92F7
:1082D00011242F933F934F935F936F937F938F93CB
:1082E0009F93AF93BF93EF93FF9382E083BD109270
:1082F000B2001CBA1DBA88EC809391018091290CC0
:108300008230C1F410921A0C1092190C10922D08A0
:1083100010922C0881E090E090931E0C80931D0C2D
:108320001092220C1092210C1092290C90931C0C8C
:1083300080931B0C8091290C813091F48091FF096E
:108340008770833039F484E690E090931A0C809320
:10835000190C04C010921A0C1092190C0E94C34000
:108360008AE08093280CFF91EF91BF91AF919F918C
:108370008F917F916F915F914F913F912F910F90CE
:108380000FBE0F901F9018951F920F920FB60F926D
:1083900011240F900FBE0F901F9018951F920F92EF
:1083A0000FB60F9211240F900FBE0F901F901895CB
:1083B0001F920F920FB60F9211242F933F934F935A
:1083C0005F936F937F938F939F93AF93BF93EF933D
:1083D000FF938091190C90911A0C019690931A0CAE
:1083E0008093190C8091290C8230C9F410921A0CD8
:1083F0001092190C10922D0810922C0881E090E038
:1084000090931E0C80931D0C1092220C1092210C44
:108410001092290C90931C0C80931B0C0DC0809122
:10842000190C90911A0C885E9340BCF010921A0CB3
:108430001092190C0E94C3408091280C882331F0BF
:108440008091280C81508093280C07C08091930163
:10845000873019F486E080939301FF91EF91BF91EB
:10846000AF919F918F917F916F915F914F913F91CC
:108470002F910F900FBE0F901F9018951F920F9283
:108480000FB60F9211248F939F938091D4029091F5
:10849000D50201969093D5028093D40280919101E8
:1084A000882359F0809191018150809391018091AE
:1084B0009101882311F481E08DBB9F918F910F90E2
:1084C0000FBE0F901F9018951F920F920FB60F922C
:1084D00011248F939F93EF93FF938091C00090910D
:1084E000C6008C7179F480912004E82FF0E0E15E01
:1084F000FC4F90838F5F80932004809121048F5FD5
:1085000080932104FF91EF919F918F910F900FBE67
:108510000F901F9018951F920F920FB60F92112473
:108520002F938F939F93EF93FF9320911C0322230C
:10853000B9F090911B03E92FF0E0E552FD4F8081E7
:108540008093C6009F5F90931B03822F815080937E
:108550001C03882329F48091C1008F7D8093C10082
:10856000FF91EF919F918F912F910F900FBE0F90E0
:108570001F9018951F920F920FB60F9211248F9390
:1085800080911C03882349F48091C1008F7B8093E4
:10859000C10010921E0310921D038F910F900FBE09
:1085A0000F901F901895CF93DF93EC0163E37BE06E
:1085B00044E050E00E949663892B11F481E017C0DB
:1085C000CE016FE27BE043E050E00E949663892B8E
:1085D00011F482E00CC0CE0168E27BE046E050E09E
:1085E0000E949663892B11F483E001C080E0DF9143
:1085F000CF910895CF93DF93019719F0C0E0D0E0B9
:1086000005C083E59DE00E94CE18EC0187E39DE064
:108610000E94CE189E01280F391FC901DF91CF910A
:108620000895A0E0B0E0E7E1F3E40C9421633B019E
:10863000E82FFF27E7FDF095EE0FFF1FED53F84FF2
:108640004590549086EF9DE00E94CE184C01C201E7
:108650000E94CE18EC0188ED9DE00E94CE185C01CE
:10866000C2010E94CE186C018AEB9DE00E94CE18D8
:108670007C01C2010E94CE188C0186EA9DE00E9416
:10868000CE18C80DD91DCA0DDB1DCC0DDD1DCE0DBC
:10869000DF1DC00FD11FC80FD91F81E068167104FC
:1086A000A9F486E99DE00E94CE187C01C2010E94D7
:1086B000CE188C018BE79DE00E94CE189701200F09
:1086C000311F2C0F3D1F280F391F07C086E79DE083
:1086D0000E94CE189C012C0F3D1FC901CDB7DEB7FB
:1086E000E0E10C943D63EF92FF920F931F93182FDC
:1086F00086E390E00E949C168EED91E00E94CE18D9
:108700007C01E12FFF27E7FDF095EE0FFF1FE35CF3
:10871000F74F859194910E94CE188C018CE09EE0D9
:108720000E94CE180E0D1F1D080F191FC8011F91A2
:108730000F91FF90EF900895A0E0B0E0E2EAF3E43B
:108740000C942763082F86E390E00E949C168EED20
:1087500091E00E94CE185C01C02FDD27C7FDD095A7
:10876000CC0FDD1FFE01E35CF74F859194910E94D1
:10877000CE188C0188E49EE00E94CE186C01FE01A8
:10878000ED53F84F859194910E94CE187C018AE3B5
:108790009EE00E94CE180A0D1B1D0C0D1D1D0E0D16
:1087A0001F1D080F191FC801CDB7DEB7EAE00C94F2
:1087B0004363AF92BF92CF92DF92EF92FF920F93FB
:1087C0001F938C01F62EE72E89ED9CE00E94CE18B7
:1087D0005C01C8010E94CE188C018FEC9CE00E94C5
:1087E000CE186C01EF2DFE2DDF010D900020E9F772
:1087F0001197AE1BBF0B8F2D9E2DBD010E94011640
:108800007C0184EC9CE00E94CE180A0D1B1D0C0D0F
:108810001D1D0E0D1F1D080F191FC8011F910F915F
:10882000FF90EF90DF90CF90BF90AF900895A4E0BD
:10883000B0E0EDE1F4E40C942F63BE016F5F7F4F75
:108840000E94D73CCE01029662E070E00E940116C1
:108850002496E2E00C944B63A8E0B0E0E2E3F4E499
:108860000C9423637C01FC0180819181BE016F5FC8
:108870007F4F0E94F33CCE01029664E070E00E94BC
:1088800001163C018FE20E94CA15F70182810E9405
:1088900017448C018FE20E94CA15F70183810E9460
:1088A00017444C0180E20E94CA15F70184810E949E
:1088B00017445C018AE30E94CA15F70185810E9472
:1088C00017446C018AE30E94CA15F70186810E9451
:1088D0001744080D191D0B5F1F4F0A0D1B1D0C0DB2
:1088E0001D1D080F191F060D171DC8012896EEE063
:1088F0000C943F63A8E0B0E0E0E8F4E40C941F635C
:108900006C0180E39DE00E94CE189E838D83F6016A
:10891000808191810E94CE188C0182E19DE00E94AD
:10892000CE1898878F83F601828193810E94CE189A
:108930001C0189E09DE00E94CE182C01F601848183
:108940007E010894E11CF11CB7010E94D73CF7019D
:1089500001900020E9F73197EE19FF09BF010E944D
:1089600001163C018BEF9CE00E94CE184C01F601F1
:108970008581B7010E94D73CF70101900020E9F7FB
:108980003197EE19FF09BF010E9401165C0181EFCA
:108990009CE00E94CE187C01F60186819781FC0143
:1089A000DF010D900020E9F71197AE1BBF0BBD0151
:1089B0000E9401162D813E81020F131FEF81F88561
:1089C0000E0F1F1F020D131D040D151D060D171D83
:1089D000080D191D0A0D1B1D0E0D1F1D080F191F57
:1089E000C8012896E2E10C943B63A8E2B0E0EBEF0B
:1089F000F4E40C942B63082F112707FD1095000F4A
:108A0000111FF801E75DFB4F85919491F801E45B3C
:108A1000FE4F4591549139E0E32EF12CEC0EFD1EF2
:108A2000B7010E94581CF801EF5DFB4F85919491AE
:108A30009A838983F801E750FC4F859194919C8338
:108A40008B8381E28D838FE18E83F886EF82CE0166
:108A500001960E947A44A896E6E00C944763A8E148
:108A6000B0E0E5E3F5E40C942B63E82EFF24E7FC8B
:108A7000F0948701000F111FF801ED56FC4F85910E
:108A8000949101C0A895F999FDCF0E9433649B0190
:108A9000AC012F3F8FEF38078FEF48078FEF580754
:108AA00059F4F701EE0FFF1FEE0FFF1FE356FC4FC7
:108AB0002591359145915491F801ED51FC4F8591E7
:108AC00094919A838983F801E757FC4F859194919B
:108AD0009C838B8382E18D838FE08E83CA01B901F1
:108AE000AE01475F5F4F0E94453F98878F83CE015D
:108AF00001960E947A446896E6E00C944763A0E0F1
:108B0000B0E0E5E8F5E40C9427635C0180E00E94A6
:108B10009C436C0180E00E942F45EC0181E00E94A3
:108B20002F457C0182E00E942F458C0183E00E944A
:108B30002F45CC0DDD1DCE0DDF1DC00FD11FC80F81
:108B4000D91F81E0A816B10419F48DE093E002C0AA
:108B500085E493E00E94CE18C80FD91F81E090E011
:108B60000E94FA426091800570918105C80FD91F5B
:108B700088E1AE010E944C23CDB7DEB7EAE00C9449
:108B80004363AAE9B0E0E7ECF5E40C941F639C01B1
:108B9000880F991FBC01F3E0660F771FFA95E1F784
:108BA000680F791F665A7A4F70938105609380052C
:108BB000F901EA57F84FE081E13009F070C6232B44
:108BC00029F0E2E88E2EE6E09E2E04C072E8872EA1
:108BD00075E0972EC4016AE879E00E94A463FC0165
:108BE000108263ECE62E67E0F62E00E0F701659157
:108BF0007491C40146E050E00E949663892B09F409
:108C000055C00F5F22E030E0E20EF31E063071F730
:108C100086E390E00E949C168EED91E00E94CE18B3
:108C20002C018EEA99E00E94CE18480E591E882425
:108C300099248EE999E00E94CE185C01F401ED536D
:108C4000F84F859194910E94CE188C018AE999E0A1
:108C50000E94CE186C01F401E35CF74F859194916A
:108C60000E94CE187C0181E999E00E94CE180A0D7D
:108C70001B1D0C0D1D1D0E0D1F1D080F191F400E75
:108C8000511E42E050E0840E951E5CE08516910472
:108C900081F680E090E00E94FA4260918005709138
:108CA0008105480E591E88E1A2010DC657E0452EE8
:108CB000512C480C591C002309F043C0D4011796CD
:108CC0008C91882319F480E090E038C000E010E037
:108CD0006E010894C11CD11C46E0842E912C800E9C
:108CE000911EF401E757FC4F65917491C2010E94F7
:108CF000A4637C01009701F10396B6010E94E13E56
:108D0000813079F4F401ED56FC4F8591949101C0C6
:108D1000A895F999FDCF49815A816B817C810E9488
:108D200061640894E108F108F701108202501040D4
:108D3000FFEF083F1F0781F681E090E00E947F452A
:108D4000C4C5013009F081C0D2018C91882319F487
:108D50008824992459C0DE011C96E4EAF1E088E0F9
:108D600001900D928150E1F732E1832E912C8C0E0F
:108D70009D1E00E010E02CE3C22ED12CCC0EDD1E97
:108D800090E2B92E86E0282E312C200E311EF10102
:108D9000E750FC4F65917491C2010E94A4637C016D
:108DA000009779F1F6012B2D11922A95E9F7BC0174
:108DB0006D5F7F4FC6010E94FF63D4018D919C912E
:108DC000B6010E94FF63F101E75DFB4F659174916D
:108DD00001C0A895F999FDCFC60140E250E00E947C
:108DE0003F640894E108F108F70110820250104036
:108DF0002EEF3FEF820E931E3FEF083F130709F05F
:108E0000C1CFB1E08B2E912C81E00E949C436C017C
:108E100080E00E94F5442C0181E00E94F5447C0131
:108E200082E00E94F5448C0183E00E94F5444C0CE2
:108E30005D1C4E0C5F1C400E511E480E591E41E039
:108E40008416910409F07FC07BC0023009F08FC006
:108E5000D2018C91882319F48824992445C0C20139
:108E600067EC79E00E94A4637C010097D1F105963C
:108E70000E94983D90933308809332088F5F9F4FF4
:108E800031F4109233081092320801C0A895F99974
:108E9000FDCF609132087091330884EC90E00E941D
:108EA0006D640894E108F108F7011082C20164ECD6
:108EB00079E00E94A4630097A1F00396BE016F5F62
:108EC0007F4F0E94E13E813061F401C0A895F9997D
:108ED000FDCF49815A816B817C8180EC90E00E94BA
:108EE0006164A1E08A2E912C82E00E949C436C0177
:108EF00084E00E942F452C018CEC99E00E94CE1852
:108F00007C018E010C5E1F4F8091320890913308D6
:108F1000B8010E94F33CF80101900020E9F7319775
:108F2000E01BF10BC801BF010E9401164C0C5D1C37
:108F30004E0C5F1C480E591EF1E08F16910419F477
:108F40008DE093E002C085E493E00E94CE187C019E
:108F5000E40CF51C81E090E00E94FA4260918005EB
:108F600070918105E80EF91E88E1A701ACC40330B9
:108F700009F04FC1C2010E94D342813019F4F8E0D8
:108F8000FF2E05C0823011F40E943C50FF2483E084
:108F90000E9473438C0189E39AE00E94CE1860918D
:108FA000800570918105080F191F88E1A8010E94B2
:108FB0004C23882309F089C486E390E00E949C1624
:108FC0006F2CAA24BB24ECE22E2E312C2C0E3D1E3D
:108FD0002F2D285FC656DF4F2883CA59D040E62D73
:108FE000F0E074E0EE0FFF1F7A95E1F7DE015C968A
:108FF000E75EF54F80E101900D928150E1F7DBA033
:109000004C8C5D8C3E8DCE57DF4F3883C258D0409C
:109010004F8DCF57DF4F4883C158D04058A1C0581B
:10902000DF4F5883C058D04079A0CAA08CA09DA023
:109030008EA19FA1C258DF4F99838883CE57D0401D
:1090400080E19BE00E94CE188C016394862D0E94E3
:1090500017447C0186E09BE00E94CE18E00EF11ED2
:10906000E80EF91E8D2D81508330D8F45E824D823A
:10907000CE57DF4F9881C258D0409F83CF57DF4FE4
:10908000A881C158D040A887C058DF4FB881C058C8
:10909000D040B9877A86CB86CE0105960E942C44B3
:1090A00004C08FEF9AE00E94CE18E80EF91E85EFFB
:1090B0009AE00E94CE182701480E591EE2E0DE1603
:1090C00061F486EE9AE00E94CE187C0189ED9AE068
:1090D0000E94CE18E80EF91E77C0F1E0DF1609F005
:1090E0006EC021E982162EE7920644F08CEC9AE0DD
:1090F0000E94CE187C01E40CF51C5AC097FC02C0FB
:109100008BE201C08DE20E94CA15C40197FE03C024
:10911000909581959F4FB1010E94F33CF101019020
:109120000020E9F73197E219F309C101BF010E945C
:1091300001164C0187EC9AE00E94CE186C01C258CF
:10914000DF4F48815981CE57D04057FD02C08BE296
:1091500001C08DE20E94CA15C258DF4F88819981F3
:10916000CE57D04097FF03C0909581959F4FB10196
:109170000E94F33CF10101900020E9F7E219F309A4
:109180003397CE018E96BF010E9401168C0183ECAD
:109190009AE00E94CE1862E0E62EF12CE40CF51C59
:1091A000E80CF91CEC0CFD1CE00EF11EE80EF91E9B
:1091B00080EB9AE00E94CE18E80EF91E07C080EA04
:1091C0009AE00E94CE187C01E40CF51C85E99AE037
:1091D0000E94CE18E80EF91EAE0CBF1CC656DF4F1B
:1091E0005881CA59D040651609F0F9CE60918005C2
:1091F0007091810588E1A5010E944C23882309F024
:1092000064C386E390E00E949C1683E060E070E017
:1092100098C1043009F09DC1C2010E94D34281303F
:1092200039F488E0C856DF4F8883C859D0400DC054
:10923000823019F40E94315003C0833009F4179A28
:10924000C856DF4F1882C859D04084E00E9473434B
:109250008C0188E39BE00E94CE186091800570919C
:109260008105080F191F88E1A8010E944C2388235B
:1092700009F02BC386E390E00E949C16C956DF4F8D
:109280001882C759D040EE961FAE1EAEEE9754E13D
:10929000252E312C2C0E3D1E8EEC9BE00E94CE180C
:1092A0008C01C956DF4FE881C759D040C856DF4FFF
:1092B0009881C859D040E90FF0E044E0EE0FFF1F5D
:1092C0004A95E1F7CF01875E944FDC011C962D9102
:1092D0003D914D915C911F97CD56DF4F2883398387
:1092E0004A835B83C359D0401A96CC901A971B9639
:1092F000BC91C756DF4FB883C959D040DF01AF5D7D
:10930000B44FEC901196DC90DC0116966C91169798
:1093100015965C91DF01A35EB44F7C91DC0113963E
:109320004C911397E55EF44FE0812D913C9111979C
:109330001796FC90FF2009F4CAC08F2D815084300D
:1093400028F48AEB9BE00E94CE180BC03E832D834D
:10935000EF83488779875A876B87CE0105960E94ED
:109360002C44080F191F80EB9BE00E94CE182C01A3
:10937000EF2DF0E0EE0FFF1FEC5BF84F859194911D
:109380000E94CE18400E511E480E591EB5E0FB1625
:1093900009F03FC08AEA9BE00E94CE183C018E2D66
:1093A0009D2DB1010E945F3CF10101900020E9F781
:1093B0003197E219F309C101BF010E9401164C0166
:1093C00084EA9BE00E94CE185C018C2DC756DF4FCB
:1093D0009881C959D040B1010E945F3CF1010190D0
:1093E0000020E9F73197E219F309C101BF010E949A
:1093F00001166C018DE99BE00E94CE187C01CD56D0
:10940000DF4F88819981C359D040B1010E945F3CF0
:1094100041C0EAE0FE1621F0F7E0FF1609F05EC059
:1094200086E99BE00E94CE183C018E2DB1010E947E
:10943000473CF10101900020E9F73197E219F30967
:10944000C101BF010E9401164C018FE89BE00E9400
:10945000CE185C018C2DB1010E94473CF1010190B6
:109460000020E9F73197E219F309C101BF010E9419
:1094700001166C0187E89BE00E94CE187C01CD5656
:10948000DF4F688179818A819B81C359D040A101D6
:109490000E94893CF10101900020E9F73197E2191F
:1094A000F309C101BF010E9401168C0189E20E94EB
:1094B000CA150894411C511C460C571C480C591CD9
:1094C0004A0C5B1C4C0C5D1C4E0C5F1C05C081E7FC
:1094D0009BE00E94CE182C01400E511E86E69BE0B8
:1094E0000E94CE18480E591EEE962EAD3FADEE9757
:1094F000240D351DEE963FAF2EAFEE97C956DF4FC8
:109500003881C759D0403F5FC956DF4F3883C759AC
:10951000D040383009F0C0CE60918005709181054F
:1095200088E1EE964EAD5FADEE970E944C23882306
:1095300009F0CBC186E390E00E949C1684E061E0D4
:1095400070E00E9411438C0181E090E00E94FA4299
:1095500098C1053009F09EC185E00E947343CF5643
:10956000DF4F99838883C159D04086E99CE00E94EF
:10957000CE188C0160914505709146058091470594
:10958000909148052CE3E22EF12CEC0EFD1EA70174
:109590000E94453FBC018BE89CE00E94D943CD5717
:1095A000DF4F99838883C358D040609149057091FB
:1095B0004A0580914B0590914C05A7010E94453FBB
:1095C000BC018FE79CE00E94D943CB57DF4F9983C2
:1095D0008883C558D04060914D0570914E058091AB
:1095E0004F0590915005A7010E94453FBC018FE6B1
:1095F0009CE00E94D943C957DF4F99838883C7589D
:10960000D0406091F9097091FA098091FB0990911D
:10961000FC09A7010E94453FBC0184E69CE00E9432
:10962000D943C757DF4F99838883C958D04087E50E
:109630009CE069EE79E00E94D943C557DF4F9983DA
:109640008883CB58D0408091FF09E82FF0E0E77085
:10965000F070EE0FFF1FEB55F74F65917491C70146
:109660000E94866388E49CE0B7010E94D943C357F7
:10967000DF4F99838883CD58D04080919301E82FA4
:10968000F0E0EE0FFF1FEA58F64F65917491C701A5
:109690000E9486638CE39CE0B7010E94D943C157C6
:1096A000DF4F99838883CF58D04080910001B70164
:1096B0000E94473C80910101BE01625C7F4F0E9485
:1096C000473CB7016C5F7F4F809102010E94473C8D
:1096D0008DE2FE01EE5BFF4F8083B701695F7F4F34
:1096E000809103010E94473CB701675F7F4F8091E3
:1096F00004010E94473CB701655F7F4F80910501DF
:109700000E94473CFE01E75BFF4F108280E39CE034
:10971000B7010E94D9431C012091B304822F6AE053
:109720000E94C262805D8CAF822F0E94C262905DF7
:109730009DAF1EAE8EE19CE0B7010E94D9432C0183
:10974000C7016CE770E00E9486638DE09CE0B70182
:109750000E94D9433C018090080A9090090AA09089
:109760000A0AB0900B0AC501B4012CE330E040E0D6
:1097700050E00E940463CA01B901A7010E94723D32
:109780007CE5C72ED12CCC0EDD1EB7016B5F7F4F61
:10979000C6010E94FF63C60167E07CE00E9472631D
:1097A000C501B4012CE330E040E050E00E940463C6
:1097B000DC01CB01B7010E94F33CC601BE01615C34
:1097C0007F4F0E94E063C60162E07CE00E9472630A
:1097D00083EF9BE0B6010E94D9436C0186EE9BE0CB
:1097E0000E94CE187C0181E090E00E94FA42CF56A0
:1097F000DF4F48815981C159D040040F151FCD5703
:10980000DF4FA881B981C358D0400A0F1B1FCB5727
:10981000DF4FE881F981C558D0400E0F1F1FC9578F
:10982000DF4F28813981C758D040020F131FC75717
:10983000DF4F48815981C958D040040F151FC557C3
:10984000DF4FA881B981CB58D0400A0F1B1FC357E7
:10985000DF4FE881F981CD58D0400E0F1F1FC1574F
:10986000DF4F28813981CF58D040020F131F020DDE
:10987000131D040D151D060D171D0C0D1D1D0E0DC0
:109880001F1D6091800570918105080F191F88E1E7
:10989000A80119C0609180057091810511C0E23066
:1098A00079F486E390E00E949C168DE691E00E9498
:1098B000CE18AC01609180057091810588E103C0EC
:1098C00081E140E050E00E944C23C656DF4FE2E1C8
:1098D0000C943B63682F88E046E753E10E94BB1A73
:1098E0000895E82FF0E0EE0FFF1FE65CFF4E459174
:1098F000549180E061E00E94BB1A0895E82FF0E0E7
:10990000EE0FFF1FE357F04F4591549180E060E068
:109910000E94BB1A0895A0E1B0E0E1E9FCE40C94D8
:109920002963E090080AF090090A00910A0A109150
:109930000B0AC801B7012CE330E040E050E00E9480
:109940000463CA01B9016E010894C11CD11CA601AF
:109950000E94723D80E061E0AE014A5F5F4F0E946D
:10996000CB1AC801B7012CE330E040E050E00E9480
:109970000463DC01CB01B6010E94F33C8AE061E0A4
:10998000AE014C5F5F4F0E94CB1A6096E8E00C94EA
:109990004563A4E0B0E0EFECFCE40C942763B82E40
:1099A000A62E6A01FA0180817E010894E11CF11C57
:1099B000B7010E94D73C8E010E5F1F4F8B2D6A2D81
:1099C000A8010E94CB1A8AE30E94621AF6018181E3
:1099D000B7010E94D73CC8010E94691A8AE30E941D
:1099E000621AF6018281B7010E94D73CC8010E9429
:1099F000691A2496EAE00C944363A3E0B0E0E3E044
:109A0000FDE40C942A63D82E7A018B0140348EE752
:109A1000580785E0680780E0780738F088E06D2D0A
:109A20004DE653E10E94BB1A2EC0CB01BA0120E1E2
:109A30003EE040E050E00E9404632983C801B70182
:109A400020E13EE040E050E00E940463162F072F23
:109A5000F82EE92E2CE330E040E050E00E94046351
:109A60002A83612F702F8F2D9E2D2CE330E040E054
:109A700050E00E9404636B8388E06D2DAE014F5F60
:109A80005F4F0E94C94C2396E7E00C944663809197
:109A90007008813049F44091690850916A086091DA
:109AA0006B0870916C081BC08731E1F480916508E8
:109AB00090916608A0916708B09168088F5F9F4FEA
:109AC000AF4FBF4F19F4EAE7F0E115C040915D08D0
:109AD00050915E0860915F087091600881E00E947B
:109AE000FD4C0895883119F4E8E7F0E104C08931AC
:109AF00039F4E6E7F0E14591549188E061E004C073
:109B000088E061E046E753E10E94BB1A0895A3E2B2
:109B1000B0E0EDE8FDE40C942663082F0E948A1A59
:109B2000093018F4402F4F5C02C0402F49508FE09D
:109B300060E00E94D61AE02FF0E044E0EE0FFF1F35
:109B40004A95E1F7DE011496E75EF44F80E101905B
:109B50000D928150E1F7DB849E81CF809884A984A7
:109B6000BA848D2D8150843068F18D2D85508232DC
:109B700048F534E1E32EF12CEC0EFD1E892FB701E0
:109B80000E94D73C8E010B5E1F4F80E060E0A80171
:109B90000E94CB1A8FE20E94621A8C2DB7010E949C
:109BA000D73CC8010E94691A80E20E94621A998219
:109BB000AA82BB8286E060E0AE014F5F5F4F0E94E9
:109BC000C94C06C080E060E042E553E10E94BB1A48
:109BD000ED2DF0E0EE0FFF1FEC5FFC4E4591549130
:109BE00080E061E00E94BB1AA396EBE00C94426314
:109BF000A3E2B0E0EEEFFDE40C942563182F0E9481
:109C00008A1A8BE00E947E4CE12FF0E064E0EE0FB8
:109C1000FF1F6A95E1F7DE011496E75EF54F80E1DC
:109C200001900D928150E1F7DB84CE80BF80888463
:109C30009984AA8454E1E52EF12CEC0EFD1E812FAF
:109C40008F5FB7010E94D73C8E010B5E1F4F8EE0E5
:109C500060E0A8010E94CB1A80E061E00E94921AA5
:109C60008D2D8150823068F58C2DB7010E94D73C34
:109C7000C8010E94691A8FE20E94621A8B2DB701F7
:109C80000E94D73CC8010E94691A80E20E94621AB1
:109C900089829A82AB8286E061E0AE014F5F5F4FBE
:109CA0000E94C94C80E20E94621A82E0D81611F428
:109CB00082E404C081E0D81651F482E50E94621A61
:109CC00006C080E061E042E553E10E94BB1AA39622
:109CD000ECE00C944163A3E1B0E0E1E7FEE40C9416
:109CE000236380910D0AE82FF0E0EE0FFF1FEC5682
:109CF000FF4E65917491CE0108960E948663609034
:109D000041017090430180904501A0904D01B090B9
:109D10004E010091490110914A010F5F1F4F909031
:109D2000470180914B0190914C01FCE0CF2ED12C4A
:109D3000CC0EDD1E8459984FB6010E94F33CEDE035
:109D4000EE2EF12CEC0EFD1E80E060E0A7010E94DB
:109D5000CB1A8FE20E94621A802FB6010E94D73C74
:109D6000C7010E94691A8FE20E94621A892DB6010A
:109D70000E94D73CC7010E94691A80E20E94621AC1
:109D80008E010C5F1F4FAA0CBB1CAA0CBB1C8FE5DD
:109D90009EE0A80EB91EC801B5010E948663C801E5
:109DA0000E94691A80E20E94621A0091FF090770FE
:109DB00091F480910601803C11F481E415C0803457
:109DC00011F489E411C0803811F484E40DC080914D
:109DD0000C08805D09C0013011F482E505C0023035
:109DE00011F08AE401C087E40E94621A89827A82B3
:109DF0006B8280E061E0AE014F5F5F4F0E94C94C13
:109E000080E20E94621ACE0108960E94691A80E2DE
:109E10000E94621A023060F480910701BE016C5FFB
:109E20007F4F0E94D73CCE0105960E94691A21C03F
:109E30000230C9F48091FF09887321F486E40E94FE
:109E4000621A0FC0883011F482E503C0803189F4B2
:109E50008AE50E94621A8091FF0986FF02C082E5AE
:109E600006C086E404C080E30E94621A81E30E9477
:109E7000621AE0919301F0E0E558F14FE4918E2FE2
:109E80000E94621A6396EEE00C943F63A0E1B0E09A
:109E9000ECE4FFE40C9429630091FD090E948A1A06
:109EA000002319F40E946B4ED8C0013019F580E0F0
:109EB00060E041E40E94D61A609145057091460524
:109EC00080914705909148058E010F5F1F4FA801B3
:109ED0000E94453F0E94691A80E061E04DE40E94C3
:109EE000D61A6091490570914A0580914B05909171
:109EF0004C0524C0023041F580E060E047E40E9458
:109F0000D61A60914D0570914E0580914F05909144
:109F100050058E010F5F1F4FA8010E94453F0E9410
:109F2000691A80E061E044E40E94D61A6091F90960
:109F30007091FA098091FB099091FC09A8010E9497
:109F4000453F0E94691A89C0033079F581E00E947B
:109F50007E4C8091B3046AE00E94C262805D0E94E0
:109F6000621A8091B3046AE00E94C262892F805D08
:109F70000E94621A83E00E94714C04E0B0E0EB2E74
:109F8000B1E0FB2E6E010894C11CD11CF701819138
:109F90007F01B6010E94473CAC01802F61E00E9426
:109FA000CB1A0E5F003191F758C0043061F480E0A5
:109FB00060E049EE59E00E94CB1A84E00E94714CA7
:109FC0000E94474D4AC0053091F586E00E947E4CC4
:109FD0008091FF098770823031F0813021F08091CB
:109FE0000E0A882391F188E060E046E753E10E9481
:109FF000BB1A85E00E94714C809132089091330821
:10A00000892B71F080910F0A9091100A019741F409
:10A010000E94AA0EAB01BC0181E00E94FD4C1DC054
:10A0200088E061E046E753E10E94BB1A16C00630A3
:10A03000A1F48CE00E947E4C85E061E041E653E1B2
:10A040000E94BB1A0E948B4C08C00E94C50EAB0137
:10A05000BC0180E00E94FD4CCCCF6096E8E00C94FF
:10A06000456380E091E0E9E1FBE0DF019C011D92A6
:10A0700021503040E1F7089580E091E0E9E1FAE015
:10A08000DF019C011D9221503040E1F70895EF92CD
:10A09000FF920F931F93182F89E29BE069E17BE009
:10A0A00040EF50E00E94C763609127017091280142
:10A0B000E0912501E0902301F090210100911F0122
:10A0C000F0911D01153079F44091AD045091AE042A
:10A0D0002091AB043091AC048091A9049091AA0422
:10A0E000A0E0B0E032C01A3011F0173089F480914E
:10A0F0005405482F50E080915505282F30E080917D
:10A10000560590915705A0915805B09159051DC06D
:10A11000812F8850823048F080E090E0A0E0B0E0ED
:10A1200020E030E040E050E010C04091C604509183
:10A13000C7042091C4043091C5048091BC0490915F
:10A14000BD04A091BE04B091BF048093250B9093F1
:10A15000260BA093270BB093280B3093240B20934E
:10A16000230B5093220B4093210B1093200BF09361
:10A170001F0B00931E0BF0921D0BE0921C0BEF5F68
:10A18000E0931B0B6459784F70931A0B6093190B73
:10A190001A3079F01B3169F0113259F01C3049F056
:10A1A0001D3039F0113029F0123019F0143009F057
:10A1B00017981F910F91FF90EF900895FF920F93C2
:10A1C0001F93F82E89E29AE08C0100511040B801EB
:10A1D00040EF50E00E94C7638091270190912801D1
:10A1E0008459984F509125015F5FB0912301A09150
:10A1F0002101F0911F01E0911D0160910E08709105
:10A200000F08209110083091110840910D0810920C
:10A21000280A1092270A1092260A4093250AF092E3
:10A22000200A3093240A2093230A7093220A609311
:10A23000210AE0931F0AF0931E0AA0931D0AB0930F
:10A240001C0A50931B0AF801918380831F910F9180
:10A25000FF9008951F93CF93DF93EC01162F109278
:10A26000290C1E860C960E94983D8E3391050CF0A9
:10A2700066C090937801809377011C86CE010A9680
:10A280000E94983D8C3391050CF059C090937A014F
:10A29000809379011A86CE0108960E94983D8831F4
:10A2A00091050CF04CC090937C0180937B01188643
:10A2B000CE0106960E94983D009709F440C0803276
:10A2C0009105ECF590937E0180937D011E82CE0175
:10A2D00004960E94983D01978C30910584F59093E7
:10A2E000800180937F011C82CE010E94983D8C5694
:10A2F0009740909382018093810110928401109283
:10A300008301109286011092850187E791E00E94F7
:10A310004A1E6093230C7093240C8093250C909319
:10A32000260C8091230C9091240CA091250CB091C7
:10A33000260CB7FD02C01093290C81E001C080E01B
:10A34000DF91CF911F910895AF92BF92CF92DF928C
:10A35000EF92FF920F931F93379B08C01092120A3F
:10A360001092110A89E0809393017AC18091930140
:10A37000893019F482E08093930110910E0A112321
:10A3800009F46EC11130D9F41092290C0E949C1B63
:10A390008091110A9091120A892B19F483EA93E1B2
:10A3A00002C08CE993E10E94C51C82E080930E0AF2
:10A3B0000E94631B9093140A8093130A51C11230B8
:10A3C000D9F50E94B01B813009F034C18091110A87
:10A3D0009091120A892BC1F482E294E066E973E15C
:10A3E00045E050E00E949663892B39F481E090E0CB
:10A3F0009093120A8093110A11C080E490E00E94A9
:10A40000E20E1093930113C182E294E06DE873E1D0
:10A4100048E050E00E949663892B11F483E052C01B
:10A42000A3E5B1E0EDE1F1E082E101900D92815010
:10A43000E1F710920E0A15C1133041F40E949C1BE3
:10A4400086E893E10E94C51C84E0B0CF143009F087
:10A4500051C00E94B01B813009F03FC010922C0403
:10A460008AE294E00E94983D009779F1803291054C
:10A4700064F590937E0180937D011092290487E218
:10A4800094E00E94983D01978C309105F4F49093EC
:10A49000800180937F011092260482E294E00E9462
:10A4A000983D8C56974097FD10C090938201809301
:10A4B0008101109284011092830110928601109202
:10A4C000850185E080930E0ACBC080E490E00E9475
:10A4D000E20E81E080939301AAC00E94631B209149
:10A4E000130A3091140A821B930B805D974008F485
:10A4F000B7C0ABC0153041F40E949C1B8FE793E1BD
:10A500000E94C51C86E052CF163009F0A9C00E94F7
:10A51000B01B813009F08EC010922A0488E294E0CA
:10A520000E94983D8C3391050CF081C09093780186
:10A53000809377011092270485E294E00E94983D71
:10A540008C3391050CF073C090937A01809379015C
:10A550001092240482E294E00E94983D8831910593
:10A560000CF065C090937C0180937B0187E791E0BC
:10A570000E944A1E7B018C0180E7A82E81E8B82E3C
:10A580008FEFC82E8FEFD82EEA0CFB1C0C1D1D1D63
:10A5900017FD48C0F89420918D0130918E014091B3
:10A5A0008F0150919001789480911B0190911C0132
:10A5B000892B01F580913708909138080097D1F0E8
:10A5C00057016801A21AB30AC40AD50AA601950167
:10A5D000D7FE07C050954095309521953F4F4F4F7E
:10A5E0005F4FA0E0B0E082179307A407B50714F40B
:10A5F00082E019C0E092230CF092240C0093250C09
:10A600001093260C81E08093290C1092110810926F
:10A61000100810920F0810920E08109293011092D9
:10A62000920105C081E0809393010E94B60B1092C5
:10A630000E0A16C00E94631B2091130A3091140A5F
:10A64000821B930B805D974058F080E490E00E945D
:10A65000E20E83E08093930110920E0A85E201C01E
:10A6600080E01F910F91FF90EF90DF90CF90BF900F
:10A67000AF900895A1E0B0E0E0E4F3E50C94256329
:10A68000182F0E949C1B183019F48FEF93E106C01D
:10A69000103111F0CC244BC08BEC93E10E94C51C0F
:10A6A0000E94631B5C018C01CC24DD244E010894C4
:10A6B000811C911C02C0DD2487010E94631B7C0168
:10A6C0000817190709F0A895C7018A199B09805D29
:10A6D000974018F025E2C22E2AC0DD2059F4C401AB
:10A6E0000E94801B813041F78981843229F7DD2463
:10A6F000D394E2CF81E0D81669F40E94B01BC82E33
:10A7000021E0821719F492E0D92ED6CF82E0C81644
:10A7100099F60DC022E0D21679F682E294E06DEB54
:10A7200073E14DE050E00E949663892B21F68C2D59
:10A730002196ECE00C944163FC01808191819A3276
:10A7400039F09A3029F03196992311F08927F6CF04
:10A750000E94473C0895A5E1B0E0E1EBF3E50C94DD
:10A760002B638091A5049091A604892BD1F4CE018E
:10A7700001960E94801B813009F0BCC1898184321E
:10A7800009F0B8C10E94631B9093A4048093A304B2
:10A7900081E090E09093A6048093A5041092A20417
:10A7A000A9C10E94B01B813009F093C11091FF092B
:10A7B000187309F058C082E294E062EB73E14AE05A
:10A7C00050E00E949663892B09F094C190912D046A
:10A7D000993331F481E380932B0490932C0406C0C9
:10A7E00082E380932B0480E380932C048BE294E03B
:10A7F00062E070E00E942A51813009F05CC1F89457
:10A8000010921A0C1092190C8091230C9091240C28
:10A81000A091250CB091260C8093260890932708D0
:10A82000A0932808B093290880938D0190938E01FE
:10A83000A0938F01B0939001789480913A04813372
:10A8400011F484E0D5C0823321F485E08093930134
:10A85000D8C0833309F04EC180913C04803309F0A5
:10A8600030C186E0C5C082E294E0BE016E5F7F4FDA
:10A870000E949C5382E294E06AE270E00E94EB63E3
:10A88000FC0191818A81981709F036C192818B81F0
:10A89000981709F031C182E294E06CEA71E044E07B
:10A8A00050E00E940664009731F48091FF098068AF
:10A8B0008093FF091FC1183009F0A6C084E294E01C
:10A8C0006EEA73E143E050E00E949663892B09F041
:10A8D00011C182E294E06CE270E00E94EB630097A9
:10A8E00009F4C4C08C010F5F1F4FCE010E96B80152
:10A8F00046E050E00E941464C8016CE270E00E94DF
:10A90000EB63FC01009709F4B1C0F18001966CE2A1
:10A9100070E00E94EB63009709F4A8C001966CE216
:10A9200070E00E94EB63009709F4A0C001966CE20E
:10A9300070E00E94EB63009709F498C001966CE206
:10A9400070E00E94EB63009709F490C001966CE2FE
:10A9500070E00E94EB63009709F488C001966CE2F6
:10A9600070E00E94EB63009709F480C001966CE2EE
:10A9700070E00E94EB638C01009709F477C0BC0182
:10A980006F5F7F4FCE010C9642E050E00E9414644E
:10A99000B8016D5F7F4FCE010A9642E050E00E9401
:10A9A0001464B8016B5F7F4FCE01089642E050E01F
:10A9B0000E941464F8018581873324F081E38E833B
:10A9C00089E303C082E38E8380E38F83CE01069602
:10A9D00061E070E00E942A51882309F46CC0F1E420
:10A9E000FF1609F46AC026E5F21609F03FC088E0B8
:10A9F000809393018091020A9091030A892B09F4B4
:10AA000065C00E94B60B76C0103109F073C084E2B5
:10AA100094E06AEA73E143E050E00E949663892B78
:10AA200009F068C088E08093930182E294E06CE2D0
:10AA300070E00E94EB630097B9F08C010F5F1F4F2D
:10AA400036E0E32EF12CEC0EFD1ECE010E96B80181
:10AA500046E050E00E941464C8016CE270E00E947D
:10AA6000EB638C01009721F40E94B60B83E245C092
:10AA70000F5F1F4FCE010C96B80142E050E00E94DC
:10AA800014640D5F1F4FCE010A96B80142E050E0FA
:10AA90000E9414640D5F1F4FC701B80144E050E0ED
:10AAA0000E941464C70161E070E00E942A5188236B
:10AAB00021F40E94B60B82E220C08091280C8823EA
:10AAC00011F087E001C086E080939301109292011B
:10AAD00011C00E94631B2091A3043091A404821B27
:10AAE000930B885E934030F01092A6041092A50458
:10AAF00085E203C080E001C084E26596E6E00C9444
:10AB00004763A8E0B0E0E7E8F5E50C942B6381E04B
:10AB10000E94B51A81E061E042EF56E10E94BB1A43
:10AB20008091020A9091030A7E010894E11CF11CB5
:10AB3000B7010E94F33CAC0186E061E00E94CB1AB1
:10AB400086E061E0A70125E000E010E00E941240ED
:10AB5000892B19F421E030E012C0C7010E94983D12
:10AB6000BC019093030A8093020A01C0A895F99949
:10AB7000FDCF82ED90E00E946D6420E030E0C901DD
:10AB80002896E6E00C944763A8E0B0E0EAECF5E52F
:10AB90000C942B6381E00E94B51A81E061E040E0F3
:10ABA00057E10E94BB1A8091000A9091010A7E0130
:10ABB0000894E11CF11CB7010E94F33CAC0186E053
:10ABC00061E00E94CB1A86E061E0A70125E000E089
:10ABD00010E00E941240892B19F421E030E012C0ED
:10ABE000C7010E94983DBC019093010A8093000A1E
:10ABF00001C0A895F999FDCF80ED90E00E946D64A9
:10AC000020E030E0C9012896E6E00C9447631F93EA
:10AC1000182F0E948A1AE12FF0E0EE0FFF1FE25C6E
:10AC2000FA4E4591549180E060E00E94BB1A1F915A
:10AC30000895EF92FF921F93DF93CF930F92CDB7BA
:10AC4000DEB780E10E9407561091180AE12FF0E06C
:10AC5000EE0FFF1FE353F94E4591549180E061E000
:10AC60000E94BB1A7E010894E11CF11C812F63E055
:10AC7000A7010E94EF3F182F8981893159F1843152
:10AC8000C9F41093180A01C0A895F999FDCF8CE377
:10AC900090E00E943964682F01C0A895F999FDCF12
:10ACA0009C7F192B8CE390E0712F0E946D6420E053
:10ACB00030E012C081E00E94B51AE12FF0E0EE0F03
:10ACC000FF1FE353F94E4591549180E061E00E94EB
:10ACD000BB1ACCCF21E030E0C9010F90CF91DF91BA
:10ACE0001F91FF90EF900895EF92FF921F93DF93D3
:10ACF000CF930F92CDB7DEB78FE00E940756109129
:10AD0000A704E12FF0E0EE0FFF1FEE56F94E45913C
:10AD1000549180E061E00E94BB1A7E010894E11C1E
:10AD2000F11C812F67E0A7010E94EF3F182F898156
:10AD3000893109F45CC0843109F049C01093A7043B
:10AD40008091FF098770823079F51092C10011233C
:10AD500019F484E395E01DC0113019F48AE992E0FA
:10AD600018C0123019F48CE491E013C0133019F4B8
:10AD700085EA90E00EC0143019F482E590E009C035
:10AD8000153019F489E290E004C0163031F48BE1FB
:10AD900090E09093C5008093C40088E98093C1003F
:10ADA0008091C60001C0A895F999FDCF86E090E09A
:10ADB0000E943964792F01C0A895F999FDCF86E0EA
:10ADC00090E0612F0E946D6420E030E012C081E0CD
:10ADD0000E94B51AE12FF0E0EE0FFF1FEE56F94E7C
:10ADE0004591549180E061E00E94BB1A9ACF21E026
:10ADF00030E0C9010F90CF91DF911F91FF90EF904C
:10AE00000895A8E0B0E0E7E0F7E50C942B638EE04E
:10AE10000E94075681E061E043ED56E10E94BB1AB3
:10AE200080913708909138087E010894E11CF11C4C
:10AE3000B7010E94F33CAC0187E061E00E94CB1AAD
:10AE400087E061E0A70125E000E010E00E941240E9
:10AE5000892B19F421E030E012C0C7010E94983D0F
:10AE6000BC01909338088093370801C0A895F999E0
:10AE7000FDCF88EC90E00E946D6420E030E0C901D5
:10AE80002896E6E00C944763A8E0B0E0EAE4F7E532
:10AE90000C942B638DE00E94075681E061E042EE46
:10AEA00056E10E94BB1A80913008909131087E01D2
:10AEB0000894E11CF11CB7010E94F33CAC0189E04D
:10AEC00061E00E94CB1A89E061E0A70125E000E083
:10AED00010E00E941240892B19F421E030E012C0EA
:10AEE000C7010E94983DBC019093310880933008BF
:10AEF00001C0A895F999FDCF86EC90E00E946D64A1
:10AF000020E030E0C9012896E6E00C944763EF9218
:10AF1000FF921F93DF93CF930F92CDB7DEB78CE0F4
:10AF20000E9407568091FF0990E076E096958795FC
:10AF30007A95E1F7182F1170E12FF0E0EE0FFF1F67
:10AF4000E15EF94E4591549180E061E00E94BB1AA8
:10AF50007E010894E11CF11C812F62E0A7010E9490
:10AF6000EF3F182F89818931A1F1843111F501C09A
:10AF7000A895F999FDCF8CE390E00E943964209167
:10AF8000FF09112331F42F7B2093FF09BC01677F58
:10AF900007C020642093FF09BC01686001C0A89528
:10AFA000F999FDCF8CE390E00E946D6420E030E0E1
:10AFB00012C081E00E94B51AE12FF0E0EE0FFF1FF2
:10AFC000E15EF94E4591549180E061E00E94BB1A28
:10AFD000C3CF21E030E0C9010F90CF91DF911F91E5
:10AFE000FF90EF900895EF92FF921F93DF93CF931E
:10AFF0000F92CDB7DEB78BE00E9407561091FF0984
:10B000001695169516951770E12FF0E0EE0FFF1FBD
:10B01000EB5FF94E4591549180E061E00E94BB1ACC
:10B020007E010894E11CF11C812F63E0A7010E94BE
:10B03000EF3F182F8981893109F43AC0843141F5F5
:10B0400001C0A895F999FDCF8CE390E00E94396486
:10B05000BC01687F8091FF09877C112319F48093DC
:10B06000FF090DC0113029F488608093FF096160E9
:10B0700006C080618093FF09626001C0A895F999BC
:10B08000FDCF8CE390E00E946D6420E030E012C0C0
:10B0900081E00E94B51AE12FF0E0EE0FFF1FEB5F99
:10B0A000F94E4591549180E061E00E94BB1ABCCFFB
:10B0B00021E030E0C9010F90CF91DF911F91FF9007
:10B0C000EF900895CF92DF92FF920F931F93DF933B
:10B0D000CF930F92CDB7DEB788E00E940756F0906D
:10B0E0000D0AEF2DF0E0EE0FFF1FEA54FA4E4591E6
:10B0F000549180E061E00E94BB1A6E010894C11C6B
:10B10000D11C8F2D66E0A6010E94EF3FF82E8981A9
:10B11000893109F434C00F2D10E0843109F5F09223
:10B120000D0AF801EE0FFF1FEE0FFF1FEE53FA4E50
:10B1300085919591A591B4918093890190938A010D
:10B14000A0938B01B0938C0101C0A895F999FDCF14
:10B150008CEC90E0B8010E946D6420E030E011C0FA
:10B1600081E00E94B51AF801EE0FFF1FEA54FA4E73
:10B170004591549180E061E00E94BB1AC2CF21E06A
:10B1800030E0C9010F90CF91DF911F910F91FF9097
:10B19000DF90CF900895CF92DF92FF920F931F938D
:10B1A000DF93CF930F92CDB7DEB787E00E940756AB
:10B1B00001C0A895F999FDCF8AEC90E00E9439640E
:10B1C0008C01FF24F394F822EF2DF0E0EE0FFF1F27
:10B1D000E15BF94E4591549180E061E00E94BB1A19
:10B1E0006E010894C11CD11C8F2D62E0A6010E9443
:10B1F000EF3FF82E8981893191F1843101F58091F9
:10B20000FF09982F9770FF2031F4B8016E7F9130BD
:10B2100061F4887F06C0B8016160992331F4887FAA
:10B2200081608093FF0901C0A895F999FDCF7F77D0
:10B230008AEC90E00E946D6420E030E012C081E072
:10B240000E94B51AEF2DF0E0EE0FFF1FE15BF94E03
:10B250004591549180E061E00E94BB1AC5CF21E086
:10B2600030E0C9010F90CF91DF911F910F91FF90B6
:10B27000DF90CF900895A8E0B0E0E1E4F9E50C9408
:10B280002B6386E00E94075680E061E04EE057E1C4
:10B290000E94BB1A80913208909133087E01089475
:10B2A000E11CF11CB7010E94F33CAC0189E061E0B4
:10B2B0000E94CB1A89E061E0A70125E000E010E0E0
:10B2C0000E941240892B19F421E030E012C0C7011E
:10B2D0000E94983DBC01909333088093320801C0CE
:10B2E000A895F999FDCF84EC90E00E946D6420E070
:10B2F00030E0C9012896E6E00C944763A4E1B0E091
:10B30000E4E8F9E50C9429636B010E94075601C03B
:10B31000A895F999FDCFC6010E94336469837A83A9
:10B320008B839C8345E0E42EF12CEC0EFD1EA701DF
:10B330000E94453F81E061E0A7012FE000E010E0BE
:10B340000E941240892B19F421E030E015C0C7019A
:10B35000BE016F5F7F4F0E94E13E813059F401C012
:10B36000A895F999FDCF49815A816B817C81C601ED
:10B370000E94616420E030E0C9016496E8E00C942A
:10B38000456385E060EC70E00E947E59089583E09B
:10B390006CE270E00E947E59089582E068E270E0FD
:10B3A0000E947E59089581E064E270E00E947E5917
:10B3B000089580E060E270E00E947E590895CF9287
:10B3C000DF92FF920F931F93DF93CF930F92CDB72E
:10B3D000DEB784E00E94075601C0A895F999FDCF19
:10B3E0008CE090E00E9439648C01F12EFF1CFF2458
:10B3F000FF1CEF2DF0E0EE0FFF1FEE5CF94E4591C4
:10B40000549180E061E00E94BB1A6E010894C11C57
:10B41000D11C8F2D62E0A6010E94EF3FF82E89819A
:10B42000893141F18431B1F4FF2029F41092700880
:10B43000B8017F7706C080937008B801706801C0BA
:10B44000A895F999FDCF8CE090E00E946D6420E012
:10B4500030E012C081E00E94B51AEF2DF0E0EE0F4F
:10B46000FF1FEE5CF94E4591549180E061E00E942F
:10B47000BB1ACFCF21E030E0C9010F90CF91DF910F
:10B480001F910F91FF90DF90CF900895A4E0B0E05E
:10B49000ECE4FAE50C942E63182F0E948A1A80E0DF
:10B4A00060E042E257E10E94BB1AE12FFF27E7FD6F
:10B4B000F095EE0FFF1FE25CFA4E4591549180E04B
:10B4C00061E00E94BB1A812F8F5FBE016F5F7F4FCB
:10B4D0000E94D73C8BE060E0AE014E5F5F4F0E9460
:10B4E000CB1A8DE060E04EE157E10E94BB1A249632
:10B4F000E3E00C944A63CF92DF92FF920F931F9385
:10B50000DF93CF93CDB7DEB7A3970FB6F894DEBF26
:10B510000FBECDBFDE011296E1EBF1E082E20190B9
:10B520000D928150E1F70E94465AFF246E01089463
:10B53000C11CD11C8F2D62E1A6010E94EF3FF82EA5
:10B5400089818931C1F0843119F000E010E00EC02A
:10B5500081E1F81681F0EF2DF0E0EE0FFF1FEC0D0A
:10B56000FD1D0180F281E02D09958C018F2D0E9437
:10B57000465A012BF9F280917008882309F045C0E2
:10B58000109272081092710880E290E044E651E057
:10B5900068EA70EC0E949E1C609345057093460516
:10B5A000809347059093480584E290E040E05FEF88
:10B5B0006FEF7FEF0E949E1C6093490570934A05D0
:10B5C00080934B0590934C0588E290E041E051E078
:10B5D00068EA70EC0E949E1C60934D0570934E05C6
:10B5E00080934F05909350058CE290E041E051E04C
:10B5F00068EA70EC0E949E1C6093F9097093FA0946
:10B600008093FB099093FC0917C08431A9F481E071
:10B6100090E09093720880937108A8E0B1E0EDE1AA
:10B62000F1E082E101900D928150E1F70E94C32880
:10B63000882311F00E944750A3960FB6F894DEBFFE
:10B640000FBECDBFCF91DF911F910F91FF90DF9083
:10B65000CF900895EF92FF920F93DF93CF93CDB7E2
:10B66000DEB760970FB6F894DEBF0FBECDBFA82F30
:10B67000002309F461C07E010894E11CF11C88E0FC
:10B68000F70111928A95E9F729833A834B835C830A
:10B690006D837E83AF83988780E2801BE82FFF272E
:10B6A000E7FDF09549815A816B817C81181684F001
:10B6B00019861A861B861C86882799278E1B9F0B46
:10B6C00004C0440F551F661F771F8A95D2F728C004
:10B6D000202F332727FD3095DB01CA01022E04C03D
:10B6E000880F991FAA1FBB1F0A94D2F789879A87D0
:10B6F000AB87BC8704C07695679557954795EA95C3
:10B70000D2F78D819E81AF81B88504C0880F991FC3
:10B71000AA1FBB1F2A95D2F7482B592B6A2B7B2BCC
:10B720004D875E876F87788B29853A854B855C8549
:10B730006D857E85AF8598898A2F60960FB6F894BF
:10B74000DEBF0FBECDBFCF91DF910F91FF90EF9085
:10B750000895EF92FF920F93DF93CF93CDB7DEB7AB
:10B7600060970FB6F894DEBF0FBECDBFA82F0023A1
:10B7700009F467C07E010894E11CF11C88E0F70120
:10B7800011928A95E9F729833A834B835C836D8311
:10B790007E83AF83988780E2801B4D815E816F81BD
:10B7A0007885E82FFF27E7FDF0951816B4F0DB0148
:10B7B000CA01BB0F880B982FDC018D879E87AF874E
:10B7C000B88B882799278E1B9F0B04C075956795AA
:10B7D000579547958A95D2F728C0202F332727FD04
:10B7E0003095DB01CA01022E04C0B595A795979547
:10B7F00087950A94D2F78D879E87AF87B88B04C050
:10B80000440F551F661F771FEA95D2F789819A81E9
:10B81000AB81BC8104C0B695A795979587952A956D
:10B82000D2F7482B592B6A2B7B2B49875A876B877A
:10B830007C8729853A854B855C856D857E85AF85BE
:10B8400098898A2F60960FB6F894DEBF0FBECDBFE1
:10B85000CF91DF910F91FF90EF900895AEE5B0E0AA
:10B86000E4E3FCE50C941F63A8E04E010894811CFE
:10B87000911CF4016A2E11926A94E9F729833A83A4
:10B880004B835C836D837E838F839887CE0109967B
:10B89000FC011192AA95E9F7A986BA86CB86DC86C7
:10B8A000ED86FE860F87188B29843A844B845C844E
:10B8B000ED84FE840F85188969807A808B809C8056
:10B8C0006DA67EA68FA698AA6D807E808F809884B4
:10B8D000E114F1040105110509F0B3C36214730406
:10B8E0008404950408F03DC100E0201600E0300615
:10B8F00001E0400600E0500688F41FEF21163104F5
:10B900004104510439F030F048E0E42EF12C012DCF
:10B91000112D18C0EE24FF24870114C020E0221648
:10B9200020E0320620E0420621E0520630F038E105
:10B93000E32EF12C012D112D05C020E1E22EF12C7A
:10B94000012D112DD201C1010E2C04C0B695A79571
:10B95000979587950A94D2F78D529E4FDC012C91D2
:10B9600080E290E0A0E0B0E08E199F09A00BB10B3F
:10B970007C018D01E21AF10801091109E114F104B9
:10B9800001051105A1F10E2C04C0220C331C441C2E
:10B99000551C0A94D2F7A40193010E2C04C0220F67
:10B9A000331F441F551F0A94D2F780E290E08E198E
:10B9B0009F096DA47EA48FA498A804C09694879430
:10B9C000779467948A95D2F7622A732A842A952AF3
:10B9D000ADA4BEA4CFA4D8A804C0AA0CBB1CCC1C88
:10B9E000DD1CEA94D2F7ADA6BEA6CFA6D8AA620106
:10B9F000EE24FF24CDAADEAAEFAAF8AE92018101BF
:10BA00002070307009AF1AAF2BAF3CAFC401B30147
:10BA1000A70196010E94E2627B018C01C401B3017F
:10BA20002DA93EA94FA958AD0E94E262C901DA01D1
:10BA30003C014D01C401B30129AD3AAD4BAD5CAD44
:10BA40000E94A3629B01AC018701FF24EE24ADA4F8
:10BA5000BEA4CFA4D8A8C601AA27BB275701680156
:10BA6000A82AB92ACA2ADB2AA216B306C406D50612
:10BA7000E0F408946108710881089108A20CB31CD5
:10BA8000C41CD51CA214B304C404D50470F0A216BF
:10BA9000B306C406D50648F4089461087108810805
:10BAA0009108A20CB31CC41CD51CA21AB30AC40A68
:10BAB000D50AC601B5012DA93EA94FA958AD0E94CE
:10BAC000E2627B018C01C601B5012DA93EA94FA9F7
:10BAD00058AD0E94E262C901DA015C016D01C60144
:10BAE000B50129AD3AAD4BAD5CAD0E94A3629B019F
:10BAF000AC018701FF24EE248DA59EA5AFA5B8A9B2
:10BB0000A070B070E82AF92A0A2B1B2BE216F30664
:10BB100004071507C0F40894A108B108C108D108AA
:10BB2000E20CF31C041D151DE214F30404051505B5
:10BB300050F0E216F3060407150728F40894A1084C
:10BB4000B108C108D108D30199278827860175015A
:10BB5000E82AF92A0A2B1B2BE9AAFAAA0BAB1CAB81
:10BB6000CFC4211431044104510471F461E070E048
:10BB700080E090E020E030E040E050E00E94E262AF
:10BB8000C901DA011C012D0100E0201600E0300699
:10BB900001E0400600E0500688F41FEF2116310452
:10BBA0004104510431F028F048E050E060E070E0DA
:10BBB00017C040E050E060E070E012C020E02216C4
:10BBC00020E0320620E0420621E0520628F048E15B
:10BBD00050E060E070E004C040E150E060E070E000
:10BBE000D201C101042E04C0B695A79597958795FB
:10BBF0000A94D2F78D529E4FDC012C91E0E2EE2E9A
:10BC0000F12C012D112DD801C701841B950BA60B1A
:10BC1000B70B821B9109A109B1090097A105B105D4
:10BC200061F464015301A218B308C408D50831E0D7
:10BC3000632E712C812C912C1EC16F968FAF6F9744
:10BC4000082E04C0220C331C441C551C0A94D2F745
:10BC5000EE2DE81B640153010E2E04C0D694C79448
:10BC6000B794A7940A94D2F7A40193016F960FACEE
:10BC70006F9704C0220F331F441F551F0A94D2F739
:10BC80006DA47EA48FA498A80E2E04C096948794C9
:10BC9000779467940A94D2F784017301E22AF32A15
:10BCA000042B152BE9A6FAA60BA71CA732018824A2
:10BCB0009924920181012070307021960CAF1DAF44
:10BCC0002EAF3FAF2197C601B501A40193010E9499
:10BCD000E2627B018C01C601B501A40193010E94BF
:10BCE000E262C901DA0125968CAF9DAFAEAFBFAF5E
:10BCF0002597BC01CD0121962CAD3DAD4EAD5FAD7C
:10BD000021970E94A3629B01AC018701FF24EE24CE
:10BD1000A9A4BAA4CBA4DCA4C601AA27BB275C01B2
:10BD20006D01AE28BF28C02AD12AA216B306C406C8
:10BD3000D50660F525966CAD7DAD8EAD9FAD259792
:10BD4000615070408040904025966CAF7DAF8EAFC3
:10BD50009FAF2597A20CB31CC41CD51CA214B3041E
:10BD6000C404D50498F0A216B306C406D50670F430
:10BD7000615070408040904025966CAF7DAF8EAF93
:10BD80009FAF2597A20CB31CC41CD51CA21AB30AE2
:10BD9000C40AD50AC601B501A40193010E94E2625A
:10BDA0007B018C01C601B501A40193010E94E262EE
:10BDB000C901DA013C014D01C401B30121962CAD4A
:10BDC0003DAD4EAD5FAD21970E94A3629B01AC01DA
:10BDD0008701FF24EE2489A59AA5ABA5BCA5A07078
:10BDE000B07057016801A82AB92ACA2ADB2AA2160C
:10BDF000B306C406D506E0F408946108710881080A
:10BE00009108A20CB31CC41CD51CA214B304C40416
:10BE1000D50470F0A216B306C406D50648F40894FB
:10BE20006108710881089108A20CB31CC41CD51CC0
:10BE30008DA59EA5AFA5B8A96F960FAC6F9704C04E
:10BE4000880F991FAA1FBB1F0A94D2F78DA79EA720
:10BE5000AFA7B8ABA21AB30AC40AD50A2596ECACB0
:10BE6000FDAC0EAD1FAD2597D70199278827682A0D
:10BE7000792A8A2A9B2A82012227332729960CAF06
:10BE80001DAF2EAF3FAF2997A201910140705070B6
:10BE90002D962CAF3DAF4EAF5FAF2D97C601B501CC
:10BEA00029962CAD3DAD4EAD5FAD29970E94E26263
:10BEB0007B018C01C601B50129962CAD3DAD4EAD7F
:10BEC0005FAD29970E94E262C901DA0161968CAFE9
:10BED0009DAFAEAFBFAF6197BC01CD012D962CAD2C
:10BEE0003DAD4EAD5FAD2D970E94A3629B01AC01AD
:10BEF0008701FF24EE24ADA4BEA4CFA4D8A8C60118
:10BF0000AA27BB2757016801A82AB92ACA2ADB2A0F
:10BF1000A216B306C406D50660F561966CAD7DAD7C
:10BF20008EAD9FAD619761507040804090406196AA
:10BF30006CAF7DAF8EAF9FAF6197A20CB31CC41CDA
:10BF4000D51CA214B304C404D50498F0A216B306F9
:10BF5000C406D50670F461507040804090406196F0
:10BF60006CAF7DAF8EAF9FAF6197A20CB31CC41CAA
:10BF7000D51CA21AB30AC40AD50AC601B50129966E
:10BF80002CAD3DAD4EAD5FAD29970E94E2627B01C5
:10BF90008C01C601B50129962CAD3DAD4EAD5FAD0E
:10BFA00029970E94E262C901DA015C016D01C601B4
:10BFB000B5012D962CAD3DAD4EAD5FAD2D970E94D8
:10BFC000A3629B01AC018701FF24EE248DA59EA5F1
:10BFD000AFA5B8A9A070B070E82AF92A0A2B1B2BCC
:10BFE000E216F30604071507C0F40894A108B10887
:10BFF000C108D108E20CF31C041D151DE214F30462
:10C000000405150550F0E216F3060407150728F499
:10C010000894A108B108C108D1086196ECACFDAC48
:10C020000EAD1FAD6197D70199278827960185012D
:10C03000082B192B2A2B3B2B09AB1AAB2BAB3CAB98
:10C0400062C26E147F048006910608F451C220E09B
:10C05000E21620E0F20621E0020720E0120788F451
:10C060003FEFE316F1040105110531F028F048E037
:10C0700050E060E070E017C040E050E060E070E049
:10C0800012C040E0E41640E0F40640E0040741E05E
:10C09000140728F048E150E060E070E004C040E19F
:10C0A00050E060E070E0D801C701042E04C0B695EE
:10C0B000A795979587950A94D2F78D529E4FDC01EC
:10C0C0002C9130E2A32EB12CC12CD12CD601C5016C
:10C0D000841B950BA60BB70B821B9109A109B10913
:10C0E0000097A105B10589F4E614F70408051905C0
:10C0F00008F4F2C16DA47EA48FA498A862147304FE
:10C100008404950408F0E8C1F3C16E968FAF6E9772
:10C11000082E04C0EE0CFF1C001F111F0A94D2F75A
:10C120006A2D681BD201C101062E04C0B695A795E1
:10C13000979587950A94D2F75C016D01AE28BF28C8
:10C14000C02AD12AADA2BEA2CFA2D8A67201610197
:10C150006E960FAC6E9704C0CC0CDD1CEE1CFF1C61
:10C160000A94D2F7C9A2DAA2EBA2FCA2640153019D
:10C17000062E04C0D694C794B794A7940A94D2F715
:10C18000D401C3016E960FAC6E9704C0880F991F3F
:10C19000AA1FBB1F0A94D2F7EDA4FEA40FA518A9ED
:10C1A00004C016950795F794E7946A95D2F737017E
:10C1B0004801682A792A8A2A9B2A6D8E7E8E8F8E64
:10C1C00098A2EDA0FEA00FA118A5380188249924FB
:10C1D000980187012070307065960CAF1DAF2EAFAF
:10C1E0003FAF6597C601B501A40193010E94E262C9
:10C1F0007B018C01C601B501A40193010E94E2629A
:10C20000C901DA011C012D01C201B10165962CADF5
:10C210003DAD4EAD5FAD65970E94A3629B01AC0141
:10C220008701FF24EE24AD8CBE8CCF8CD8A0C60134
:10C23000AA27BB2757016801A82AB92ACA2ADB2ADC
:10C24000A216B306C406D50600F5089421083108E5
:10C2500041085108EDA0FEA00FA118A5AE0CBF1C0F
:10C26000C01ED11EAE14BF04C006D10670F0A216C7
:10C27000B306C406D50648F40894210831084108DD
:10C280005108AE0CBF1CC01ED11EA21AB30AC40AAC
:10C29000D50AC601B501A40193010E94E2627B01A7
:10C2A0008C01C601B501A40193010E94E262C9019B
:10C2B000DA013C014D01C401B30165962CAD3DADE1
:10C2C0004EAD5FAD65970E94A3629B01AC018701F3
:10C2D000FF24EE248D8D9E8DAF8DB8A1A070B0701F
:10C2E00057016801A82AB92ACA2ADB2AA216B3066E
:10C2F000C406D50600F50894610871088108910804
:10C300006DA17EA18FA198A5A60EB71EC81ED91E2D
:10C31000A616B706C806D90670F0A216B306C4065C
:10C32000D50648F408946108710881089108A60EA2
:10C33000B71EC81ED91ED601C501821B930BA40BC4
:10C34000B50B898F9A8FAB8FBC8FD1019927882726
:10C3500064015301A82AB92ACA2ADB2AA9AABAAABF
:10C36000CBAADCAA860175012FEF3FEF40E050E039
:10C37000E222F32204231523A601662777276D9670
:10C380004CAF5DAF6EAF7FAF6D97A9A0BAA0CBA049
:10C39000DCA06FEF7FEF80E090E0A622B722C822FA
:10C3A000D92289A19AA1ABA1BCA11D014424552485
:10C3B000C801B701A60195010E94A36269966CAFFE
:10C3C0007DAF8EAF9FAF6997C801B701A201910100
:10C3D0000E94A3623B014C016D966CAD7DAD8EADAC
:10C3E0009FAD6D97A60195010E94A3627B018C0110
:10C3F0006D966CAD7DAD8EAD9FAD6D97A201910137
:10C400000E94A3625B016C01A8019701260D371DF4
:10C41000481D591D69966CAC7DAC8EAC9FAC69977C
:10C42000C401AA27BB27280F391F4A1F5B1F2E15DF
:10C430003F054007510748F4E12CF12C61E0062F3D
:10C44000112DAE0CBF1CC01ED11ECA01AA27BB27CE
:10C45000BC01CD016A0D7B1D8C1D9D1D698C7A8CE4
:10C460008B8C9C8C661677068806990640F16615BB
:10C4700077058805990509F043C0D90199278827D0
:10C4800069962CAD3DAD4EAD5FAD69974070507073
:10C49000820F931FA41FB51F2DA53EA54FA558A918
:10C4A0006E960FAC6E9704C0220F331F441F551FAA
:10C4B0000A94D2F7281739074A075B0708F509A934
:10C4C0001AA92BA93CA9015010402040304009ABCB
:10C4D0001AAB2BAB3CAB14C066247724430121E09C
:10C4E00030E040E050E029AB3AAB4BAB5CAB0BC06B
:10C4F00066247724430119AA1AAA1BAA1CAA03C0FE
:10C50000662477244301FE01719688E0DF011D92C5
:10C510008A95E9F7A9A8BAA8CBA8DCA8A98ABA8AFB
:10C52000CB8ADC8A6D8A7E8A8F8A988E29A93A897D
:10C530004B895C89662D7E898F89988DC25ADF4F21
:10C54000E2E10C943B63629FD001739FF001829FF4
:10C55000E00DF11D649FE00DF11D929FF00D839F92
:10C56000F00D749FF00D659FF00D9927729FB00D2F
:10C57000E11DF91F639FB00DE11DF91FBD01CF0142
:10C5800011240895991B79E004C0991F961708F0AB
:10C59000961B881F7A95C9F780950895AA1BBB1B27
:10C5A00051E107C0AA1FBB1FA617B70710F0A61BB3
:10C5B000B70B881F991F5A95A9F780959095BC01D4
:10C5C000CD010895A1E21A2EAA1BBB1BFD010DC0CF
:10C5D000AA1FBB1FEE1FFF1FA217B307E407F50733
:10C5E00020F0A21BB30BE40BF50B661F771F881F0F
:10C5F000991F1A9469F760957095809590959B01A5
:10C60000AC01BD01CF01089597FB092E05260ED080
:10C6100057FD04D0D7DF0AD0001C38F45095409560
:10C62000309521953F4F4F4F5F4F0895F6F7909506
:10C630008095709561957F4F8F4F9F4F08952F92F2
:10C640003F924F925F926F927F928F929F92AF92A2
:10C65000BF92CF92DF92EF92FF920F931F93CF93EF
:10C66000DF93CDB7DEB7CA1BDB0B0FB6F894DEBF86
:10C670000FBECDBF09942A88398848885F846E84AC
:10C680007D848C849B84AA84B984C884DF80EE80F6
:10C69000FD800C811B81AA81B981CE0FD11D0FB6FF
:10C6A000F894DEBF0FBECDBFED010895911106C015
:10C6B00080538A5010F0865C06C008959927882719
:10C6C000089585FDFBCF80629111F8CF81568A5184
:10C6D000E0F708959111089581568A5108F4805227
:10C6E00085580895FB01DC010D900020E9F71197B2
:10C6F00005900D920020E1F70895FB01DC018D917A
:10C70000059080190110D9F3990B0895FB01DC0104
:10C7100005900D920020E1F70895FC01059000209E
:10C72000E9F7809590958E0F9F1F0895FB01DC011E
:10C730004150504030F08D910590801919F400203F
:10C74000B9F7881B990B0895FB0155915523A9F062
:10C75000BF01DC014D9145174111E1F759F4CD01BD
:10C760000590002049F04D9140154111C9F3FB019E
:10C770004111EFCF81E090E001970895FB01DC01CA
:10C7800002C001900D9241505040D8F708956817AB
:10C79000790768F4FB01DC01E40FF51FA40FB51F56
:10C7A00002C002900E9241505040D8F708950C9468
:10C7B000BE63DC0101C06D9341505040E0F7089525
:10C7C000FB01DC010D900020E9F7119701900D921B
:10C7D0000020E1F70895FC018191861721F088235C
:10C7E000D9F7992708953197CF010895FB01DC010E
:10C7F0008D91019080190110D9F3990B0895FB01D7
:10C80000DC0101900D920020E1F70895FB01DC01AD
:10C810004150504030F08D910190801919F4002062
:10C82000B9F7881B990B0895FB01DC01415050407A
:10C8300048F001900D920020C9F701C01D924150AF
:10C840005040E0F70895DC01CB01FC01F999FECFDF
:10C8500006C0F2BDE1BDF89A319600B40D92415088
:10C860005040B8F70895A6E1B0E044E050E00C94E1
:10C870002564A8E1B0E042E050E00C942564DC01BE
:10C88000A40FB51F4150504048F0CB01840F951FB5
:10C890002E910E94506441505040D0F70895262FA9
:10C8A000F999FECF92BD81BDF89A019700B40216A6
:10C8B00039F01FBA20BD0FB6F894FA9AF99A0FBE54
:10C8C00008950396272F0E9450640E944F64252FDD
:10C8D0000E945064242F0C9450640196272F0E94CC
:10C8E00050640C944F64DC01CB0103C02D910E9475
:10C8F0007E6441505040D0F70895262FF999FECF1D
:10C900001FBA92BD81BD20BD0FB6F894FA9AF99A6C
:10C910000FBE01960895242F0E947E64252F0E9449
:10C920007E640C9493640E947D64272F0C947E6433
:04C93000F894FFCFA9
:10C93400020000000000C010000000000900010017
:10C944000000460000000000000006010000000096
:10C954000009000100000046000000000000000083
:10C96400000000000001000000460000000000007C
:10C97400000000000000000100000046000000006C
:10C984000000000000000009000100000046000053
:10C994000000000000000000000900010000004643
:10C9A4000000000000000000000000090001000079
:10C9B400004600000000000000907E0000B469F012
:10C9C4005AC8040215CD5B07E5559A15B53B121FED
:10C9D400331349058C07AC07CC07EC07504D544B77
:10C9E40000D959D359CD59C759DF59C1593B59CBEE
:10C9F400586258C4558155F35787574457015774A3
:10CA04005619560001020203030303040404040438
:10CA140004040405050505050505050505050505C5
:10CA240005050506060606060606060606060606A5
:10CA34000606060606060606060606060606060692
:10CA44000606060707070707070707070707070775
:10CA54000707070707070707070707070707070762
:10CA64000707070707070707070707070707070752
:10CA74000707070707070707070707070707070742
:10CA84000707070808080808080808080808080825
:10CA94000808080808080808080808080808080812
:10CAA4000808080808080808080808080808080802
:10CAB40008080808080808080808080808080808F2
:10CAC40008080808080808080808080808080808E2
:10CAD40008080808080808080808080808080808D2
:10CAE40008080808080808080808080808080808C2
:10CAF40008080808080808080808080808080808B2
:04CB04000808080015
:00000001FF
